:020000040800F2
:10300000008000205FD300087D6900089D690008EA
:1030100000000000000000000000000000000000B0
:1030200000000000000000000000000077D500084C
:10303000000000000000000079D500083D030020DA
:10304000A5D30008A7D30008A9D30008ABD3000874
:10305000ADD30008AFD30008B1D30008B3D3000844
:10306000B5D3000845030020B7D30008B9D3000842
:10307000ED030020BBD30008BDD30008BFD3000878
:10308000C1D30008C9690008D9690008E9690008C6
:10309000C3D30008F9690008096A0008C5D300080D
:1030A000C7D30008C9D30008CBD3000849040020C7
:1030B000CDD30008CFD30008D1D30008D3D3000864
:1030C000014902480860704708ED00E00030000840
:1030D00000B587B054480068382108400090202887
:1030E00000D982E00098810001A040588746C04680
:1030F000EB310008EB310008EB310008EB31000840
:10310000EB310008EB310008EB310008EB3100082F
:1031100075310008EB310008EB310008EB31000895
:10312000EB310008EB310008EB310008EB3100080F
:1031300091310008EB310008EB310008EB31000859
:10314000EB310008EB310008EB310008EB310008EF
:103150007D310008EB310008EB310008EB3100084D
:10316000EB310008EB310008EB310008EB310008CF
:103170008731000830492F48086045E02E497D20FE
:103180000002086040E02C490120C00308603BE0D9
:10319000264801680322114003910068702108400D
:1031A0000009401C02900398032805D10299214888
:1031B00009F05CFE059004E002991D4809F056FEF6
:1031C0000590059A194801687F231B021940090AD6
:1031D000514305910068400F401C049005980499E4
:1031E00009F044FE144908600EE014480068072105
:1031F000C9020840C10A01208840019001990C4889
:1032000009F034FE0C490860074800680F210902E4
:10321000084081090A4840580690069A06490868FD
:10322000D040086007B000BD081002400C100240FA
:103230000024F40000127A00200500200010024053
:04324000443200080C
:10324400000000000000000000000000000000007A
:10325400000000000000000000000000000000006A
:103264000100000002000000030000000400000050
:10327400060000000700000008000000090000002C
:10328400000000000000000000000000000000003A
:103294000100000002000000030000000400000020
:1032A40010B586B0002101910591049103913A482B
:1032B40002903A4A0260012293074360031D816031
:1032C400C160540504610824446101764176827624
:1032D4000624C4611977416281622C23C25413030A
:1032E40003634263022282633C228154C16405F079
:1032F40011F8002801D002F08BFB0120039000207C
:10330400049027480590244803A905F0DBFA002817
:1033140001D002F07DFB2348039004200490002098
:1033240005901D4803A905F0CDFA002801D002F04C
:103334006FFB1D48039008200490174803A905F06B
:10334400C1FA002801D002F063FB184803900C2056
:103354000490114803A905F0B5FA002801D002F041
:1033640057FB13480390102004900B4803A905F061
:10337400A9FA002801D002F04BFB0E480390142058
:103384000490054803A905F09DFA002801D002F035
:103394003FFB06B010BDC046840E0020002401404F
:1033A40004FFFF0702000004040000080800000CEA
:0833B4008000001C400000181D
:1033BC0010B59AB01990002018901790169015908F
:1033CC00149007A8342109F0D3FD199800682D49F1
:1033DC00884255D101208003079000200F9007A848
:1033EC0007F0BEFC002801D002F00EFB2648026854
:1033FC00012109050A4302600068084006900698FE
:10340C002248026801210A430260006808400590C6
:10341C000598CF2014900320039015900020029063
:10342C00169005200190000714A906F08BFD019B56
:10343C00029A039916480490164C0460436082600B
:10344C00C2608022026101221302436192028261F6
:10345C002022C2610903016206F0E2F9002801D0C2
:10346C0002F0D2FA19980A490165199888620C2061
:10347C000090002211460BF0FFFA00980AF009FAAE
:10348C001AB010BD0024014040100240341002401C
:08349C00440F0020080002406B
:1034A40000B581B00B4800900B4901600121017106
:1034B4004171072282601022C260002202614261CF
:1034C4008261016206F04EF8002801D002F0A0FAF1
:0C34D40001B000BD681100200030024073
:1034E00082B00190019800680749884209D10748D5
:1034F0000268012109030A43026000680840009045
:10350000009802B07047C0460030024038100240B8
:1035100000B589B06846242109F030FD10481149F2
:1035200001600AF0D2F9002801D002F073FA0022FB
:10353000009201920292039204920948694606F0B1
:1035400075F8002801D002F065FA05486946102296
:1035500006F06CF8002801D002F05CFA09B000BD5A
:08356000A811002000740040D6
:1035680000B58BB00A90002009900890079006904B
:1035780005900A9800681749884228D116480268B9
:10358800012149070A430260006808400490049832
:103598001248026801210A4302600068084003904B
:1035A8000398302005900320009006900020019099
:1035B80007900520000705A906F0C6FC0099019AA6
:1035C800112002900BF05AFA02980AF064F90BB035
:1035D80000BDC046007400403C1002403410024058
:1035E80000B583B01748026801210A4302600068E9
:1035F8000840029002981448019014490160002183
:1036080041600122930383604023C36080230361E8
:1036180053024361D2028261C1610321090301623D
:1036280006F000F9002801D002F0F0F90920009016
:10363800012100220BF022FA00980AF02CF903B0BD
:1036480000BDC04638100240E80E00201C000240B1
:1036580030B593B000201290119010900F900E90FA
:103668006348026804210A430260006808400D901C
:103678000D985F48026820210A43026000680840EC
:103688000C900C985A48026801210A4302600068AD
:1036980008400B900B985648026802210A430260C2
:1036A800006808400A900A985148026808210A43AD
:1036B80002600068084009900998012461034D4898
:1036C800019022460BF05AFA0198A10300220592B4
:1036D8000BF054FA059A484807903F210BF04EFA30
:1036E800059A052000070390E50229460BF046FAE3
:1036F800059A42480490032106910BF03FFA01987D
:103708000599069A52030E920F94109111910EA9E1
:10371800089106F019FC0198059A0899E3030293A9
:103728000E930F92109206F00FFC059A07980899CD
:103738001F230E930F941092119206F005FC059A20
:1037480007980899FF231B020E930F92109406F016
:10375800FBFB0398059A089923020E930F92109287
:1037680006F0F2FB0198059A0899C0230E930F9270
:10377800109406F0E9FB0398059B069A08990E95A4
:103788000F941093119206F0DFFB029B0398059AA1
:1037980008990E930F92109406F0D6FB0498059A98
:1037A80008990E940F941092119206F0CDFB04988C
:1037B800059B069A089902250E950F94109311926D
:1037C80006F0C2FB0498059A08990C230E930F92F1
:1037D800109406F0B9FB059B069A079808992025CE
:1037E8000E950F941093119206F0AEFB13B030BDF6
:1037F800341002400008005000040050000C005033
:1038080000B599B000201890334A01211160169034
:10381800159004F0D1FC09F0D9FDFFF719FFFFF767
:10382800DFFEFFF73BFD03F0E5FAFFF737FEFFF792
:103838006BFE03F021FA00F09BFC03F0FDF903F0A6
:10384800E1F903F0B7F903F08DF903F055F900F049
:1038580097FC224807F06AFC002803D02048214939
:1038680003F0AAFB204900200AF09EFD1C481F49CE
:1038780003F05EFB1E4800681E4908401E494018B8
:10388800119011284ED81198810001A04058874600
:10389800193900082D3900082D3900082D3900087C
:1038A8002D3900082D3900082D3900082D39000858
:1038B8002D3900082D3900080F3900082D39000866
:1038C8002D3900082D3900082D3900082D39000838
:1038D80023390008053900084C1200203810002050
:1038E800B3F30008B8F30008CDF30008D2F30008DA
:1038F80000580140FF0F0000AAFBFFFFFB48FC49EE
:1039080003F016FB12E0F948FA4903F011FB0DE049
:10391800F648F94903F00CFB08E0F448F74903F0CE
:1039280007FB03E0F148F64903F002FBFE48006894
:10393800030CFE49FB4A002010900AF035FD09F0FF
:10394800ACFE02461098FA490AF02EFD03F0CEFFAD
:1039580002461098F7490AF027FD1098F649B52253
:103968000AF022FD07F030F902461098F3490AF0F0
:103978001BFD07F029F9F24988420AD8E9480F9057
:10398800F04903F019FB0F98EF4903F015FB0BF012
:1039980083F800F00DFC00F03DFC04F011FA00285B
:1039A80007D0E048E94903F0E5FA04F0C7F904F064
:1039B8008FFAE74804F030F8002803D0D948E549E1
:1039C80003F0FAFAE24804F0B3FA002803D0D54825
:1039D800E14903F0F1FADE480E9001210B02C25AC8
:1039E800521CC252DD4A11604621425A4A21415AAC
:1039F8005143DB4A1160C18F6E204843642109F0AE
:103A080031FA01460E9840228152C08BD5490222D4
:103A180009F021FD0E98408B65280ED1CC48C18A4B
:103A2800008B00044118D0480190D0480090D0483D
:103A3800D04B00220AF092FD20E0C548408B6F2849
:103A48000ED1C348C18A008B00044118C6480190B2
:103A5800C6480090C648C74B01220AF07FFD0DE01A
:103A6800BB48C18A008B00044118BF480190BF4879
:103A78000090BF48BF4B02220AF070FDBE4809F013
:103A880068FE002818D1BC4805F054FC00280ED167
:103A9800B9480AF0E9FF149014983F2108430090B0
:103AA800B649B74A9F4B00200AF07EFC03E09D48C8
:103AB800B44903F081FA03E09A48B34903F07CFA69
:103AC800B2480B9000210D9109F01EFF01460B989A
:103AD8001391102109F018FF01460D981291139BBC
:103AE800AB49904A0C920AF05FFC0C9A0D98129B15
:103AF800A8490AF059FC012000F0CAFB9E48A649D3
:103B0800062204F051FE002803D08648A34903F09A
:103B180053FAA34908680422904308609B480A9016
:103B2800002109910AF0C2FF0A98102108910AF0B1
:103B3800BDFF099B0A9819461A460BF001F8089927
:103B4800099B0A981A460AF0FBFF00F01FFC9549EA
:103B580095480860954A96491160964908609649C3
:103B68000860964908609649086096499648086032
:103B780000F02CFF7E480AF0B3FD002810D07C48E6
:103B880003F0D0FC022807D190480068002802D032
:103B980077480AF0ADFD03E0764988222220885054
:103BA8006B485421405A8A490988884206D1684995
:103BB8005222012088526C49088005E0644952224B
:103BC800002088526849088082480068002800D18F
:103BD80096E15F48008C002800D190E164482621D6
:103BE800405C002800D08AE15948008C07900128E1
:103BF8003AD00798022852D00798032800D1FBE052
:103C08000798052844D007980A2800D111E1079899
:103C1800142800D110E107981E2800D110E1079858
:103C28007D218900884200D121E107986A498842AC
:103C380000D142E107986949884200D12BE10798F1
:103C48006749884200D13CE107986649884200D11B
:103C580018E107986449884200D1F4E0079863495D
:103C6800884200D120E130E13948002103F0A6FF65
:103C7800002803D02B485E4903F09EF9344803F02E
:103C8800CBFE002803D02748324903F095F933E1E9
:103C98002448584903F04CF901F0E0FE2CE12C4887
:103CA800408B65280ED12A48C18A008B0004411830
:103CB8002D4801902D4800902D482E4B00220AF0E7
:103CC8004DFC2DE02248408B6F281BD12048C18A2B
:103CD800008B00044118244801902448009024488F
:103CE800244B01220AF03AFC1AE0C046B3F300085C
:103CF800F3F0000815F1000837F1000859F1000841
:103D08006DD30008F348C18A008B00044118F548B8
:103D18000190F5480090F548F54B02220AF01EFC88
:103D2800EAE0C046B3F3000800580140E1F5000896
:103D38007BF10008FDF50008B1F10008E3F3000885
:103D4800FF8FD00331F6000891D3000849F6000828
:103D580010130020F4F300087CEE00081412002071
:103D68001C050020000400502E14002064050020CB
:103D7800100B0020F40D0020840E002021F4000810
:103D880075F60008ABEE000842F40008A811002000
:103D980053F4000880F4000822140020D3F100082E
:103DA800080002408C1200203903002090120020E5
:103DB800ED48000888120020CC120020BC12002018
:103DC800E01200209412002069490008280500200C
:103DD800EE0500204C120020504F0000F97500003D
:103DE800C57600006E9D0000E3C4000058EC00009A
:103DF80081F30008A6F0000803F0A0FF002803D014
:103E0800B348C64903F0D8F804F062F8B14803F0A3
:103E180003FE002803D0AE48AF4903F0CDF8AD4803
:103E280004F086F8002803D0A948AC4903F0C4F888
:103E380062E002F02DFC5FE0002000F029FA5BE070
:103E480002F0C2FB58E0A348012103F0B7FE0028A6
:103E580003D09F48B04903F0AFF89E4803F0DCFD5B
:103E6800002803D09A489C4903F0A6F844E0A149E9
:103E78000A6800209060096848619649EA228852D9
:103E880002F046FD9E4800689B49884202D19C4941
:103E9800A048086030E09A4800689749884202D1F3
:103EA80097499B48086027E09548006892498842EE
:103EB80002D19349954808601EE092498E480860EF
:103EC8001AE090499048086016E095480268012178
:103ED800C943116102680021516207F075F9002891
:103EE80003D07B488F4903F067F8784900200860C1
:103EF80077488D4903F03EF876490020088402E0AF
:103F080074490020088400F023FE04F0B9F91790E2
:103F180017981699884200D12AE61798169078487B
:103F28000068804700F054FE804906910868400008
:103F38000860052000070121890309F0B0FD024649
:103F480006980168114301600068002802D017989C
:103F580000F05AFE179801F043F8179801F036FC64
:103F680017981599401A724988420FD317981590D7
:103F78005748704902F0DCFF59480068002805D00E
:103F8800544804F03FF85649002008605148808D95
:103F98000590002806D00598012804D00598022825
:103FA8002FD091E090E064480068012811D10920E1
:103FB800049009F07BFC0498694A6A491160454AF3
:103FC800EA230021D15209F066FC4C496648086092
:103FD80016E05B480068012803D148495F4808603B
:103FE8000EE058480068012803D144495A4808603F
:103FF80006E055480068012802D140495548086044
:1040080062E04D480068012803D04C480068012848
:1040180023D14F48006800281ED10920039009F0D9
:1040280045FC03984E4A4F4911602A4AEA23002169
:10403800D15209F030FC40480068012802D12F49CC
:10404800494808603D480068012802D12B49474883
:1040580008603F490120086036E0394800680128B7
:104068000AD13B480068002805D124493B4808602C
:1040780037490120086027E03248006801280AD142
:1040880033480068002805D11C4933480860304986
:104098000120086018E02C48006801280AD12C4843
:1040A8000068002805D115492A48086028490120D8
:1040B800086009E0254802681798254902910968AF
:1040C800904702990020086052E5C0464C12002033
:1040D800B3F3000810130020F4F300087CEE000886
:1040E800141200202E14002064050020100B00205C
:1040F800F40D0020A811002039030020BC12002074
:10410800E012002094120020694900081D67000889
:10411800C167000899680008D1F70008BDF00008D9
:1041280084100020F5F70008C3F5000810050020EA
:10413800C1D40100ADF4000810120020381200208C
:10414800281200202C12002024120020F412002033
:104158003412002055590008F5580008B9580008CD
:10416800741200200100002081580008B559000889
:1041780008B4024B9C4608BC6047C046390300207F
:1041880000B581B0094800908921490008F0F2FE85
:104198000099C92008800120488000208880C880B4
:1041A8000884F622885201B000BDC04610130020D2
:1041B80000B587B0164803900122019211460AF013
:1041C800DDFC019A0398022102910AF0D7FC019ABA
:1041D8000398042104910AF0D1FC7D200690C000C8
:1041E80004F054F801990398002205920AF0C6FCDD
:1041F80002990398059A0AF0C1FC03980499059A54
:104208000AF0BCFC0698800004F040F807B000BD36
:04421800000400504E
:10421C0000B583B0154800680290154801900299CA
:10422C00019A1448302309F07CFB002804D0124872
:10423C00154902F0BFFEFEE70F48104902F076FE6A
:10424C000C487D21CA00002105F034FC002804D064
:10425C0009480C4902F0AEFEFEE70748084902F097
:10426C0065FE01980149086003B000BD08ED00E04F
:10427C0000060020E80E0020B3F30008C2EE000890
:0C428C007DF600082FF20008F1F1000898
:1042980010B588B0079003F0F3FF069006982A49F6
:1042A8000968401A7D218900884202D807980028A9
:1042B80048D0264806F0DCFF2548808D002802D02B
:1042C80006982149086022490191002005908885B7
:1042D8000920029009F0EAFA019A029805991D4C02
:1042E8001D4B2360EA23D15209F0D5FA05991B4AE0
:1042F8001B4810601B4A1C4810601C4A1C48106070
:104308001C48036801220392D2431A610268516271
:1043180006F05AFF039818490B6802021A600968E8
:10432800400208600C20049002F09EF9049809F0FD
:10433800B2FA0598114908601149086011490860E6
:104348001149086008B010BD3C120020D0100020B0
:10435800101300207412002001000020CC1200204D
:104368002D5C0008BC1200207D5B00088C12002028
:10437800E95C00081C110020840E0020281200208F
:0C43880024120020101200202C12002033
:1043940000B583B001200102FA4809F082FB01282C
:1043A40040D101204102F74809F07BFB012839D1B3
:1043B40001208102F34809F074FB012832D1012065
:1043C400C102F04809F06DFB002815D1EE48EF4911
:1043D40002F0B0FDEE49EF480860EF49EF4808608D
:1043E400EF484860EF48C8608860EF4901200870D2
:1043F400EE490820488514E0E348ED4902F09AFDAF
:10440400E349EC480860E449E4480860EA48486045
:10441400E448C8608860E44901200870E34900204A
:1044240048859EE101200102D64809F03AFB0028A4
:104434003FD101204102D34809F033FB012838D190
:1044440001208102CF4809F02CFB012831D1012041
:10445400C102CC4809F025FB002815D1CA48D74928
:1044640002F068FDCA49D6480860CB49D5480860BF
:10447400D5484860CB48C8608860CB4901200870A3
:10448400CA490920488513E0F548D04902F052FD95
:10449400F549CF480860F649CA480860CD484860E5
:1044A400C048C8608860F74901200870F64948850B
:1044B40057E101200102E94809F0F3FA012840D14B
:1044C40001204102E54809F0ECFA002839D1012025
:1044D4008102E24809F0E5FA012832D10120C10243
:1044E400DE4809F0DEFA002815D1DD48F94902F06A
:1044F40021FDDD49F8480860DD49F4480860F748C3
:104504004860EC48C8608860DE4900200870DE49D5
:104514000A20488514E0D248EA4902F00BFDD2494A
:10452400E9480860D249E9480860E9484860E14838
:10453400C8608860D34900200870D34902204885A8
:104544000FE101200102C54809F0ABFA002840D16F
:1045540001204102C14809F0A4FA002839D1012000
:104564008102BE4809F09DFA012832D10120C1021E
:10457400BA4809F096FA002815D1B948CE4902F094
:10458400D9FCB949CD480860B949C8480860CC4845
:104594004860C848C8608860BA4900200870BA49B1
:1045A4000B20488514E0AE48BE4902F0C3FCAE4976
:1045B400BD480860AE49BD480860BD484860BD4874
:1045C400C8608860AF4900200870AF49032048855F
:1045D400C7E001200102A14809F063FA012842D191
:1045E400012041029D4809F05CFA01283BD10120D9
:1045F40081029A4809F055FA002834D10120C102F9
:10460400964809F04EFA002816D19548A44902F0BC
:1046140091FC95499E4808609549964808609648DB
:104624004860964888609648C8609649012008709A
:1046340095490C20488515E08948984902F07AFC90
:1046440089498A4808608A498A4808608A484860D3
:104654008A4888608A48C8608A49012008708A4963
:10466400042048857DE0012001027C4809F019FA04
:10467400002842D101204102784809F012FA0128A9
:104684003BD101208102754809F00BFA002834D18E
:104694000120C102714809F004FA002816D17048BB
:1046A4007D4902F047FC70497948086070497148B7
:1046B400086071484860714888607148C8607149F1
:1046C4000020087070490D20488515E06448714940
:1046D40002F030FC64496548086065496548086033
:1046E40065484860654888606548C8606549002039
:1046F400087065490520488533E00120C102574808
:1047040009F0CFF9002816D15548604902F012FC8F
:1047140055495F48086056495648086056484860FD
:10472400564888605648C860564901200870564962
:104734000C20488515E04A484A4902F0FBFB4A49E7
:104744004A4808604A494B4808604B4848604B480F
:1047540088604B48C8604B49012008704A490420CE
:104764004885012001033D4809F09BF9002833D115
:104774005B49012008604449488D10221043488554
:104784002DE0C04600040050B3F3000865F20008B1
:10479400F4120020295D0008CC110020F15D00080E
:1047A400315E0008390300203B0300201013002071
:1047B400F5EE0008895E0008515F00088FF20008DA
:1047C400C95F000891600008D160000820EF00086C
:1047D40029610008F16100084149002008600120B6
:1047E40041031E4809F05DF9002808D13D49012024
:1047F40008602549488D20221043488502E0394944
:10480400002008600120019001021448029005F084
:10481400EDFC01990298490205F0E8FC019902981F
:10482400890205F0E3FC01990298C90205F0DEFC57
:1048340001990298090305F0D9FC019902984903EA
:1048440005F0D4FC01990298890305F0CFFC019985
:104854000298C90305F0CAFC03B000BD000400506F
:10486400B3F30008E2F40008F4120020BD64000869
:10487400CC1100205163000895630008F16300081F
:104884004D6400083B03002010130020ADF600081F
:1048940069620008CCEF000837F30008A1EF0008B4
:1048A4000DF3000876EF0008296100089160000804
:1048B400F161000839030020E3F20008C95F000831
:1048C400D16000084BEF0008895E0008F15D000824
:1048D400515F0008B9F20008295D0008315E000844
:0848E400301200205C120020DC
:1048EC0000B583B003F0CAFC029018480068002899
:1048FC0013D1029816490968401A164988420CD3FC
:10490C0015480122019211460AF036F901980F4917
:10491C00086002980E49086015E00C4800680028F1
:10492C0011D002980A490968401A33280BD30A4857
:10493C000121002200920AF01FF900980349086037
:10494C0002980349086003B000BDC046EC12002079
:0C495C00E8120020B70300000004005027
:1049680080B512490A6800209060096848611049BA
:10497800EA2288520F491048086010480068002849
:1049880013D10F480068002808D1094911200201F5
:10499800885A401C88520B490120086008490120A8
:1049A800086003F06DFC0849086080BDA81100206C
:1049B8001013002074120020390300202812002050
:0C49C8002412002014120020140500200E
:1049D40010B586B003F056FC0146524801600068E9
:1049E40051490968401A022800D299E04D480068EC
:1049F4004D4908604D4801684D480490428F8A181B
:104A0400E8214252415EB52040004843494908F03C
:104A14000BFA01460498B5390591D822845E4649BB
:104A24000B681B1B0B60059C0B681B190B6009684A
:104A3400CB179B0CC918890B8152EA21405A0028D4
:104A44006BD03E480068002809D13C490120086029
:104A54003949002008603649D822885260E0344839
:104A6400EA21405A02282AD13148D821405E3C210B
:104A7400C943884222DC3248006800281ED109203C
:104A8400029008F015FF02982E4A136800219960DD
:104A940012685161264A0392EA23D1522A4A2B49C9
:104AA400116008F0FAFE039A254901200860872165
:104AB4004B00D15A491CD152254908602CE01C48AE
:104AC400EA21405A032827D11948D821405E3D28BD
:104AD40022DB1B48006800281ED10920009008F042
:104AE400E7FE0098174A1368002199601268516123
:104AF4000F4A0192EA23D152134A1449116008F073
:104B0400CCFE019A0E490120086087214B00D15A3E
:104B1400491CD1520E49086002E00849002008608F
:104B240006B010BD081300200C130020181200203A
:104B340010130020FF0F00000013002004130020B6
:104B44002C120020A8110020741200203903002028
:044B54001412002017
:104B580000B581B003F094FB0090009817490968EC
:104B6800401A002828D000981449086003F0A6FAD3
:104B7800082003F013FB002806D01148134902F05F
:104B8800D7F901F021FD17E0082009F0E3FD00281E
:104B980006D00B480C4902F0CBF901F079FD0BE087
:104BA800042003F0FBFA002806D00548054902F066
:104BB800BFF90020FFF76CFB01B000BD8412002094
:104BC800B3F30008F9F60008F7EF000861F30008EE
:104BD80080B508480068804707480068804707484C
:104BE8000068804706480068804706480068804794
:104BF80080BDC0468C120020901200208812002030
:084C0800CC120020BC120020B8
:104C100000B5A1B020902098CF490968401A4E28CD
:104C200000D297E12098CC490860CC481F90CC482E
:104C30001E901E9ACB49CC4B0020199009F0B8FB6E
:104C400019981F9A1E9BC949189109F0B1FB199830
:104C5000C7491A91D8228A5EC64909F0A9FB18995A
:104C600019981F9A1E9B09F0A3FB1A991998FC2208
:104C70008A5EC14909F09CFB189919981F9A1E9BDE
:104C800009F096FB1A991998EC228A5EBB4909F043
:104C90008FFB189919981F9A1E9B09F089FB1A9986
:104CA0001998CC228A5AB64909F082FB18991998AA
:104CB0001F9A1E9B09F07CFB1A991998D2228A5AD6
:104CC000B04909F075FB189919981F9A1E9B09F0B5
:104CD0006FFB1A98CA21415AAB481B90AB4A1C92F1
:104CE00000291D9001D01C981D9019981D9AA84963
:104CF00009F05EFB189919981F9A1E9B09F058FB42
:104D00001A991B98C822895A0029179001D01C981B
:104D100017901998179A9F4909F04AFB1899199802
:104D20001F9A1E9B09F044FB19989B49169109682C
:104D3000CA6A9A4909F03CFB189919981F9A1E9B58
:104D400009F036FB1699199809680A6B944909F01D
:104D50002FFB189919981F9A1E9B09F029FB1A9886
:104D6000EA21405A002802D19148159016E0804867
:104D7000EA21405A012802D18C4814900CE07C486A
:104D8000EA21415A8748884A12920229139001D099
:104D9000129813901398149014981590159A8549A9
:104DA0000020109009F004FB10981F9A1E9B6F4979
:104DB0000F9109F0FDFA6E481190E221405E0D90CE
:104DC0000A210C9108F032F80C9902460D980E92C7
:104DD0005143401A0AF042F80E9A03461098764959
:104DE00009F0E6FA0F9910981F9A1E9B09F0E0FA55
:104DF0001198F621405AC00700280CD06F490A913B
:104E0000704A00200B9009F0D3FA0A990B986C4A6B
:104E100009F0CEFA04E06949694A002009F0C8FAAD
:104E20001F9A1E9B5149002009F0C2FA5048F621F2
:104E3000405A800700280CD560490891614A00203B
:104E4000099009F0B5FA089909985F4A09F0B0FA93
:104E500004E05A495C4A002009F0AAFA1F9A1E9BF6
:104E60004249002009F0A4FA4148F621405A40077F
:104E700000280CD551490691524A0020079009F0AC
:104E800097FA06990798514A09F092FA04E04B49BB
:104E90004E4A002009F08CFA1F9A1E9B33490020CD
:104EA00009F086FA3248F621405A000700280CD54E
:104EB00042490491434A0020059009F079FA049987
:104EC0000598434A09F074FA04E03C49404A00203E
:104ED00009F06EFA1F9A1E9B2449002009F068FA17
:104EE0002348F621405A800600280CD53349029108
:104EF000344A0020039009F05BFA029903982A4A89
:104F000009F056FA04E02D49274A002009F050FA2A
:104F10001F9A1E9B1549002009F04AFA2D480121CD
:104F200008F0C1FD01280CD1244900912B4A002032
:104F3000019009F03DFA00990198294A09F038FAE0
:104F400004E01E49244A002009F032FA25490020D5
:104F500009F02EFA21B000BDDC12002011F7000884
:104F600075F600082FF50008B3F3000819F70008DC
:104F70001013002021F700082DF7000834F5000871
:104F800012F000081DF0000877F3000839F7000858
:104F90003DF5000846F50008A811002028F000089B
:104FA00033F0000844F0000847F0000841F0000822
:104FB0003EF0000879F300084FF500084AF00008B9
:104FC0004DF0000849F7000850F0000853F00008C1
:104FD00056F00008000C005061F7000851F7000877
:084FE00059F700087FF30008F7
:104FE80070B59CB012901298ED490968401AED49C5
:104FF8000968884200D8AFE31298E9490860E9498E
:1050080087200860E848C08813901399E748484308
:10501800001313901399E6484843E64907F002FF46
:105028001390E548CC21425AE4480168891A016086
:105038000068002802D5E14900200860139ADF487B
:105048000168891801600068C117490F4018C20833
:10505800D949CC200A52085AD022895A884205DDFB
:10506800D549CC20085AD02288520BE0D249CC200E
:10507800085ACE22895A884204DACF49CC20085AE5
:10508800CE228852C848408814901499C74848438B
:10509800001314901499C6484843C64907F0C2FE45
:1050A8001490C548D221425AC5480168891A01603E
:1050B8000068002802D5C24900200860149AC04838
:1050C8000168891801600068C117C90E40184209B3
:1050D800B948D2214252405ABA49884214DCBA48E7
:1050E800006800280FD1B84901200860B24AF623A9
:1050F800D15A08242143D15283214B00D15A491C4B
:10510800D152B24908600EE0AB48D221405AB049AA
:10511800884208DBAC4900200860A749F622885A73
:10512800082398438852A449D220085AD622895A7B
:10513800884205DDA049D220085AD62288520BE0C1
:105148009D49D220085AD422895A884204DA9A49B9
:10515800D220085AD4228852934801889D4848434F
:105168009D4940189D4907F05DFE9D4940181190E2
:105178009149E2200C5E9B4A13681B1B1360119C2B
:1051880013681B1913601268D317DB0ED218520963
:105198000A52085EE622895E884205DD8649E220D9
:1051A800085AE62288520BE08349E220085EE4228E
:1051B800895E884204DA8049E220085AE42288524B
:1051C8007D49E220085E098D884213DB8648006825
:1051D80000280ED1844901200860774AF623D15A65
:1051E8000143D15281214B00D15A491CD1527749F0
:1051F80008601AE07048E221415E0A91018D4B2057
:105208004843642107F02EFE01460A9888420CDACA
:1052180076480068002808D073490020086066496D
:10522800F622885A01239843885271480068012859
:1052380006D16149F622885A02231843885205E0AC
:105248005D49F622885A02239843885269480068C3
:10525800012806D15849F622885A0423184388524F
:1052680005E05549F622885A042398438852624833
:105278000068012806D15049F622885A202318438D
:10528800885205E04C49F622885A202398438852D0
:105298004948D821405E00281DD54749D820085ED6
:1052A8004042E022895A884206DD4349D820085AFC
:1052B8004042E02288520DE03F49D820085E404233
:1052C800DE22895A884205DA3B49D820085A4042EA
:1052D800DE22885218E03849D820085EDC22895A34
:1052E800884205DD3449D820085ADC2288520BE070
:1052F8003149D820085EDA22895A884204DA2E49D0
:10530800D820085ADA2288523C4B18682A49F822D1
:1053180088523B4C2068FA22885210201090394855
:105328000668394A1568AD1B15601D6813685B1956
:1053380013601268D3171B0FD21812110260334B77
:105348001E68334A1568AD1B156025681468641912
:1053580014601268D417240F121912111A60006809
:105368004C22895A884207DB26480068FD494C22AE
:10537800895A401A099001E00020099009980F9075
:10538800F9480068F7494E22895A884242DBF648B4
:105398000068F4494E22895A401A08903CE0C046F9
:1053A800AC1200204405002022140020B80B000095
:1053B800A8DE00001027000010130020E4120020CF
:1053C800480500200F270000381200201412002082
:1053D800E12E0000140500000CE3F7FFEF060000C3
:1053E800D4FEFFFFA0120020101200205C12002043
:1053F80028120020241200202C1200201C12002049
:105408002012002098120020A41200209C120020D4
:10541800A81200200020089008980E900F980E9966
:10542800401A0D900D99CE484843D04907F0FAFC30
:10543800CC490791FC2288520D9A7D208000504368
:10544800C98F07F0EFFC01460798EC228152EA2148
:10545800405A002808D1C6480068C649884203D087
:10546800C349C448086015E0BE48EA21405A0128EB
:1054780008D1BF480068C049884203D0BC49BE482B
:10548800086007E0BA480068BC49884202D0B849B9
:10549800BA480860BA480690402108F000FB014667
:1054A80006980CAA1170802108F0F9FA0BA9087067
:1054B800B448007800281AD10BA80078012804D134
:1054C800A849C8220020885203E0A649C822012022
:1054D80088520CA80078012804D1A249CA220020C9
:1054E800885203E09F49CA220120885219E00BA87C
:1054F8000078002804D19B49C8220020885203E084
:105508009849C822012088520CA80078002804D1A4
:105518009449CA220020885203E09249CA220120F5
:1055280088529048EA21405A012809D08D48EA213A
:10553800405A022804D08B48EA21405A032825D132
:105548008848D821405E032809DB8F48012211468C
:1055580009F014FB8D497D208000086015E0814822
:10556800D821405E002810DC88480068012803DB49
:1055780086490868401E086084480068002804D1ED
:1055880081480121002209F0F9FA04E07E4801214E
:10559800002209F0F3FA7E48008872494422895AA9
:1055A800884225D06F494420085A898F88421FDDD8
:1055B8006C484421405A6A49884203DB69494422BD
:1055C80067488852674805904421425A704B1A80B0
:1055D800415A66484843624907F044FC0246059828
:1055E80046214252415A4A22805A48436949086032
:1055F800694800885B494822895A88421ED0594820
:105608004821405A1E2803DC564948221F20885248
:10561800544804904821425A5F4B1A80415A5F48C7
:1056280048435F4907F0FEFB014604984A2281522D
:105638004621415A805A48435649086005200007C8
:105648000121090208F02BFA012804D14549FE225C
:105658000120885203E04349FE220020885201209D
:105668001B9000214F48405E3E494222895A884299
:1056780072D04D4809F036F93A494220085A898FC4
:10568800884203DA3749888F4222885235484221B6
:10569800405A4649884203DB324942223048885200
:1056A80030484221425A3F4B1A80002203921A92F4
:1056B800199218921792169215923D4A1592032242
:1056C800920516923B4A17921B9A531E9A4115ABA4
:1056D80002931A73415A25484843214907F0C2FBEF
:1056E80002990246039819921A902F4803F006FB74
:1056F800002801D000F08AF92F4815900320800572
:1057080016902E4817901B98411E884115A90191A3
:10571800087314484221415A14484843104907F075
:10572800A1FB0199199000201A901F4803F0E6FA8E
:10573800002801D000F06AF91B480849062203F046
:1057480033F8002803D01E481E4901F035FC1E49D5
:1057580008680422904308601CB070BD2214002021
:10576800B80B0000101300209C120020FF0F00004F
:105778008C120020E95C0008095D00086D5C0008D7
:10578800000800503B030020000C0050B01200201D
:10579800321400201C0500203414002000E204000C
:1057A80040420F0030140020840E0020B90B000086
:1057B800FFFF170004000008FFFF27004000001843
:0C57C800B3F30008D3F100080800024011
:1057D40000B583B00290192001900298204909680D
:1057E400401A0199884238D902981D490860192045
:1057F40001901C4908784000087005200007012129
:10580400C90308F04EF9002820D116480178012276
:10581400114301700078002817D01348006800284D
:1058240013D011490020086010480068002806D0F1
:105834000F49114808600D490020086005E00C4933
:105844000C48086009490120086006E00548007812
:10585400002802D104490120086003B000BDC046FD
:105864006C120020ED0500202405002028050020EE
:0C58740090120020ED480008295A00089E
:1058800000B587B00122029206926846059004A8EE
:105890000090C821018003A90191064B0B8000F004
:1058A00029F900980199029A00F006F905988546B1
:0858B00007B000BDC4090000AF
:1058B80000B587B00222029206926846059004A8B5
:1058C8000090C823038003A901910B804380064BF5
:1058D8004B8000F00BF900980199029A00F0E8F863
:0C58E8000598854607B000BDC40900000B
:1058F40000B58BB003200A906846099000200890F8
:10590400089801280CD80898420006A9C820885293
:1059140008994A0004A988520898401C0890EFE7A7
:1059240006A80190C821818004A90291074A8A80AF
:105934000322039200F0DCF801980299039A00F024
:10594400B9F8099885460BB000BDC046C4090000EB
:1059540000B58BB004200A90684609900020089096
:10596400089802280CD80898420006A9C820885232
:1059740008994A0004A988520898401C0890EFE747
:1059840006A80190C821C18004A90291074ACA80CF
:105994000422039200F0ACF801980299039A00F0F3
:1059A40089F8099885460BB000BDC046C4090000BB
:1059B40000B58DB005200C9068460B9000200A902D
:1059C4000A9803280CD80A98420007A9C8208852CC
:1059D4000A994A0004A988520A98401C0A90EFE7E1
:1059E40007A80190C821018104A90291074A0A81EC
:1059F4000522039200F07CF801980299039A00F0C2
:105A040059F80B9885460DB000BDC046C409000086
:105A140080B50248024901F0D1FA80BDB3F3000811
:045A24009BF00008EB
:105A280080B504480122114609F0A8F80249034844
:105A3800086080BD00040050901200203903002047
:105A480004490A6800209060096848610249EA220E
:0C5A580088527047A81100201013002095
:105A640000B581B011485421405A1149098888422F
:105A74000CD10E480090002102F0A2F800995620A3
:105A84000A5A0B4802800088542288520848008829
:105A9400002804D0054950220120885203E003491C
:105AA40050220020885201B000BDC04610130020CF
:045AB400EE050020DB
:105AB80000B587B0069005910492049B0698059955
:105AC80002220392054A0292019100900448054976
:105AD800054A07F0E9FC07B000BDC04600040050C5
:0C5AE800681200206412002060120020F0
:105AF40000B587B0069005910492049B0698059919
:105B040008220392054A0292019100900448054933
:105B1400054A07F0CBFC07B000BDC04600040050A6
:0C5B2400C8120020C4120020C012002093
:105B300010B58AB00422039209926846089006A81C
:105B40000190C823038004A902910B8043807D2328
:105B50009C004C80AF239B0083808C80C380064BCD
:105B6000CB80FFF7C7FF01980299039AFFF7A4FFC4
:0C5B7000089885460AB010BDC40900006A
:105B7C0000B583B00848019008210022029208F079
:105B8C00FBFF0198029A022108F0F6FF0349044832
:105B9C00086003B000BDC04600040050BC120020D9
:045BAC003903002099
:105BB00000B583B002F068FB029018480068002826
:105BC00013D1029816490968401A164988420CD325
:105BD000154810210122019208F0D4FF01980F49C5
:105BE000086002980E49086015E00C48006800281B
:105BF00011D002980A490968401AC9280BD30A48EB
:105C000010210022009208F0BDFF009803490860AF
:105C100002980349086003B000BDC046D4120020BA
:0C5C2000D01200202103000000040050FE
:105C2C0080B504481021002208F0A6FF0249034861
:105C3C00086080BD00040050CC1200203903002005
:105C4C0080B504481021012208F096FF0249034850
:105C5C00086080BD00040050CC12002039030020E5
:105C6C0000B583B002F00AFB0290184800680028C7
:105C7C0013D1029816490968401A164988420CD368
:105C8C00154804210122019208F076FF01980F4972
:105C9C00086002980E49086015E00C48006800285E
:105CAC0011D002980A490968401A33280BD30A48C4
:105CBC0004210022009208F05FFF0098034908605D
:105CCC0002980349086003B000BDC046B81200201A
:0C5CDC00B4120020B703000000040050C8
:105CE80080B504480421002208F048FF024903480F
:105CF800086080BD000400508C1200203903002089
:105D080080B504480421012208F038FF02490348FD
:105D1800086080BD000400508C1200203903002068
:105D280000B585B0049003910398002803D0284952
:105D38000220086041E0049821490968401A214975
:105D48000968884239D904981D4908601E4880218D
:105D580007F0A5FE02A908701C480078002804D1A5
:105D680002A9087842425041087002A800780190C0
:105D780001981749096888420CD001988200184890
:105D880080581449885001988100164840580D4998
:105D980008600AE0019882000E490F48885001986F
:105DA80081000E4840580749086001988100094859
:105DB8004058804701980649086005B000BDC046B4
:105DC800FC12002060050020000800503B03002062
:105DD8005C0500200412002039030020C8D1000807
:085DE800CC110020C0D100081D
:105DF00000B581B00920009007F05CFD0098074ACB
:105E000007491160074AEA230121D15207F047FDF3
:105E100005490648086001B000BDC0467412002064
:105E2000C900002010130020CC120020B15B000834
:105E300000B583B00920019007F03CFD01980C4AA1
:105E40000C4911600C4A0292EA230021D15207F05A
:105E500026FD0299094A0A4810602120C200885A8A
:105E6000401C885207490120086003B000BDC046AD
:105E7000741200201101002010130020CC12002009
:085E8000B15B000814120020C0
:105E880000B585B0049003910398002804D02849F0
:105E98000020C043086041E0049821490968401A7D
:105EA80020490968884239D904981D4908601E4864
:105EB800802107F0F4FD02A908701C48007800282A
:105EC80004D102A9087842425041087002A800781B
:105ED800019001981649096888420CDD01988200F2
:105EE8001748805813498850019881001548405830
:105EF8000C4908600AE0019882000E490E48885053
:105F0800019881000D4840580649086001988100B1
:105F180008484058804701980549086005B000BD09
:105F28008012002040050020000800503B0300209C
:105F38003C050020F411002039030020B8D10008E6
:085F4800CC110020B0D10008CB
:105F500000B585B00920019007F0ACFC0198134A08
:105F600013491160134A0392EA2300210291D1528E
:105F700007F095FC0299039881850F4A0F4810603D
:105F80000F48036801220492D2431A6102685162E9
:105F900005F01EF9039A04982121CB00D15A491C1F
:105FA000D1520849086005B000BDC04674120020F7
:105FB0000100002010130020CC1200202D5C0008EE
:085FC0001C1100201412002046
:105FC80000B585B0049003910398002803D02849B0
:105FD8000220086041E0049821490968401A2149D3
:105FE8000968884239D904981D4908601E4840212B
:105FF80007F055FD02A908701C480078002804D154
:1060080002A9087842425041087002A8007801901D
:1060180001981749096888420CD0019882001848ED
:1060280080581449885001988100164840580D49F5
:1060380008600AE0019882000E490F4888500198CC
:1060480081000E48405807490860019881000948B6
:106058004058804701980649086005B000BDC04611
:10606800F012002050050020000800503B030020DB
:106078004C050020FC11002039030020A8D100089D
:08608800CC110020A0D100089A
:1060900000B581B00920009007F00CFC0098074A79
:1060A00007491160074AEA230121D15207F0F7FBA3
:1060B00005490648086001B000BDC04674120020C2
:1060C0004100002010130020CC120020B15B00081A
:1060D00000B583B00920019007F0ECFB01980C4A51
:1060E0000C4911600C4A0292EA230021D15207F0B8
:1060F000D6FB0299094A0A48106085204200885A56
:10610000401C885207490120086003B000BDC0460A
:10611000741200208900002010130020CC120020EF
:08612000B15B0008141200201D
:1061280000B585B0049003910398002804D028494D
:106138000020C043086041E0049821490968401ADA
:1061480020490968884239D904981D4908601E48C1
:10615800402107F0A4FC02A908701C480078002818
:1061680004D102A9087842425041087002A8007878
:10617800019001981649096888420CDD019882004F
:10618800174880581349885001988100154840588D
:106198000C4908600AE0019882000E490E488850B0
:1061A800019881000D48405806490860019881000F
:1061B80008484058804701980549086005B000BD67
:1061C8007012002030050020000800503B0300201A
:1061D8002C050020EC1100203903002098D100087C
:0861E800CC11002090D1000849
:1061F00000B585B00920019007F05CFB0198134AB7
:1062000013491160134A0392EA2300210291D152EB
:1062100007F045FB0299039881850F4A0F481060EB
:106220000F48036801220492D2431A610268516246
:1062300004F0CEFF039A049885214B00D15A491CE3
:10624000D1520849086005B000BDC0467412002054
:106250000100002010130020CC1200202D5C00084B
:086260001C11002014120020A3
:1062680000B587B0069005910598002803D03049FD
:106278000420086052E0069829490968401A29490B
:10628800096888424AD90698254908602648019035
:10629800402107F004FC0146019804AA11708021EE
:1062A80007F0FDFB03A9087020480078002809D1F1
:1062B80004A9087842425041087003A9087842426C
:1062C8005041087004A80078400003A909780843E1
:1062D800029002981649096888420CD002988200F8
:1062E800174880581349885002988100154840582B
:1062F8000C4908600AE0029882000E490E4888504E
:10630800029881000D4840580649086002988100AB
:1063180008484058804702980549086007B000BD02
:10632800F812002058050020000800503B03002008
:1063380054050020DC1100203903002000D2000899
:08634800CC110020F0D1000887
:1063500000B581B00920009007F0ACFA0098084A17
:1063600008491160084AEA230121D15207F097FA3F
:10637000064907480860FFF701FC01B000BDC046B0
:10638000741200205101002010130020CC120020B4
:04639000B15B0008F5
:1063940000B583B00920019007F08AFA01980D4AEC
:1063A4000D4911600D4A0292EA230321D15207F0EC
:1063B40074FA0B490B480860FFF7DEFB02992120B1
:1063C400C200885A401C885207490120086003B063
:1063D40000BDC04674120020990100201013002053
:0C63E400CC120020B15B00081412002055
:1063F00000B583B00920019007F05CFA01980D4ABE
:106400000D4911600D4A0292EA230221D15207F090
:1064100046FA0B490B480860FFF7B0FB029985204C
:106420004200885A401C885207490120086003B086
:1064300000BDC04674120020250200201013002069
:0C644000CC120020B15B000814120020F8
:10644C0000B583B00920019007F02EFA0198104A8C
:10645C0010491160104A0292EA230021D15207F030
:10646C0018FA02990D4A0E4810600E4A0E48106038
:10647C002120C200885A401C885285204200885A2C
:10648C00401C885209490120086003B000BDC04679
:10649C0074120020B102002010130020CC12002036
:1064AC002D5C0008BC120020315B00081412002087
:1064BC0000B587B0069005910598002806D03A4A99
:1064CC000020C14311603C49086062E006983249E3
:1064DC000968401A3149096888425AD906982E49E8
:1064EC0008602F480190402107F0D7FA0146019827
:1064FC0004AA1170802107F0D0FA03A9087029486A
:10650C000078002809D104A908784242504108704B
:10651C0003A9087842425041087004A80078400052
:10652C0003A909780843029002981F490968884218
:10653C0016D021480068002811D10298012802DBEE
:10654C001D4901200860029882001C488058174998
:10655C008850029881001A484058104908600AE097
:10656C000298820011491248885002988100114803
:10657C0040580A490860029881000C48405800288D
:10658C0004D0029881000948405880470298064977
:10659C00086007B000BDC0467C1200203805002002
:1065AC00000800503B03002034050020BC110020E3
:1065BC0039030020E0D1000878120020CC11002013
:0465CC00D0D1000822
:1065D00000B583B001F058FE02901C48808D02285F
:1065E00032D01A48808D01282ED0029818490968A7
:1065F000401A1849884227D3029817490968401A57
:106600001649884220D3029815490968401A13494F
:10661000884219D3134804F02FFE02980C490860F1
:106620001148026801210191C943116102680021EA
:10663000516204F0CDFD0198044A43218B00D15AE8
:10664000491CD1520949086003B000BD1013002055
:106650003C120020E903000014050020112700006F
:1066600018050020D0100020A00F002014120020D8
:1066700081B001466846017000214056002807D4C9
:10668000684601781F2001400120884001490860C8
:0866900001B0704780E200E058
:1066980000B583B01948808D01282DD01748808D0A
:1066A800022829D016480068002825D001F0E8FD06
:1066B800144908601448026801210291C9430091F5
:1066C8001161026800210191516204F07DFD009A78
:1066D80001990E4803681A610268516204F074FD5A
:1066E8000298064A43218B00D15A491CD1520849C5
:1066F80008600C2007F0DAF803B000BD1013002082
:10670800301200203C120020EC0F0020D010002096
:046718001412002037
:10671C0000B589B00020089007901D49069105909E
:10672C0005981C49884215D81F490A680898801892
:10673C0008901E480368079AD2180792059A0B68AE
:10674C00006800901A49002007F02CFE0598401CA8
:10675C000590E5E708980E49029106F081FB029935
:10676C000D4A04924C230393D052079806F078FB01
:10677C00039A034604984E214352825A435A0749BE
:10678C00002007F00FFE06490648086009B000BD5E
:10679C0050C300004FC300001013002089F50008FF
:1067AC00E0120020390300201C12002020120020CF
:0467BC005CF5000880
:1067C00000B585B029482A4900F0B6FB01F05CFD10
:1067D0000490002003900290019001F055FD04996F
:1067E000401A2449884217D802990398401A039006
:1067F000274801680398401803900398C117090FB0
:10680000401800110290029A2249002007F0D0FDA2
:10681000012001F03FFDE0E7174800904E21415A6A
:106820000298401A0290029914484843144906F00D
:10683000FDFA014600980191019981870299C1876B
:10684000C18F6E204843642106F010FB014600987A
:1068500040228152C28F838F0A49002007F0A8FD91
:1068600009490A48086005B000BDC046B3F30008F6
:1068700059F000085FEA000010130020B80B000078
:10688000FF0F000089F70008E01200203903002004
:086890002012002069F7000846
:1068980000B583B00020029014490191009000983F
:1068A800134988420ED8184802680299891802913B
:1068B800009A03681549002007F076FD0098401CEF
:1068C8000090ECE70298094906F0CCFA014609481D
:1068D800411A094841873A21425E0849002007F0D9
:1068E80063FD07490748086003B000BD50C30000B6
:1068F8004FC30000FF07000010130020AEF500088A
:10690800E0120020390300201812002080F000084F
:10691800BFF34F8F034904480860BFF34F8F00BF90
:0C692800FDE7C0460CED00E00400FA059D
:1069340000B583B00E48026801210A430260006872
:106944000840029002980B480268012109070A4393
:106954000260006808400190019801F0C5FC022023
:1069640001F0B4FC0320400201F0C6FC03B000BDFA
:08697400401002403C100240FB
:10697C0080B504F0D5F90448022108F011F9034957
:10698C00002006F0E1FBF6E700040050A3F300083A
:10699C0000B581B006490020009006F0D5FB0098A8
:1069AC00044906F0D1FB0448022108F0F9F8FAE793
:0C69BC0015F800081DF800080004005049
:1069C80080B5024804F07AFC80BDC046EC0F002078
:1069D80080B5024804F072FC80BDC046A00F0020BC
:1069E80080B5024804F06AFC80BDC0461C11002036
:1069F80080B5024804F062FC80BDC046D01000207B
:106A080080B5024804F05AFC80BDC04684100020BE
:106A180000B583B00290029804F02AFC029800683E
:106A2800274988420BD12C49012088852B4B304AB5
:106A38001A60EA2288522B492E4808603DE00298E5
:106A4800006820490968884208D1234902208885BE
:106A5800264802680020012190472EE0029800682D
:106A680019490968884200D127E002980068174947
:106A780088421AD11849002000908885174B184A77
:106A88001A60EA2288521749174808600E48019090
:106A980004F0EEFB0099019803680122D2431A61C1
:106AA8000268516204F090FB07E002980068084908
:106AB800884202D107490120086003B000BDC046E2
:106AC80000100040A00F00201C11002000440140CD
:106AD800004801404C1200201013002074120020BE
:106AE80001000020CC1200202D5C0008F4120020C8
:086AF800F10200204D5C0008D2
:106B000000B589B000210191089107910691059186
:106B1000049103910291144801229207026041609E
:106B20008160CA43C2600161816106F0D5FF00281F
:106B300001D0FEF76FFF0120000305900A4805A968
:106B400004F0E6FC002801D0FEF764FF002002906C
:106B50000490054802A904F0A3FD002801D0FEF727
:0C6B600059FF09B000BDC04638100020ED
:106B6C0000B583B000210291019100910D480E4AAD
:106B7C000260F922426081600C4AC260816106F0B9
:106B8C00A5FF002801D0FEF73FFF002000900290E7
:106B9C000448694604F07EFD002801D0FEF734FF5E
:106BAC0003B000BDEC0F002000100040FFF9000006
:106BBC0000B583B000210291019100910D480E4A5D
:106BCC000260F922426081600C4AC260816106F069
:106BDC007DFF002801D0FEF717FF002000900290E7
:106BEC000448694604F056FD002801D0FEF70CFF5E
:106BFC0003B000BDA00F002000140040FFF90000FE
:106C0C0080B5094809490160632141600021816018
:106C1C00074AC2600161816106F058FF002801D06B
:106C2C00FEF7F2FE80BDC0461C1100200020004083
:046C3C00FFF900005C
:106C400000B581B00A4800900A4901600A494160D4
:106C500000218160094AC26001614161816106F0E1
:106C60003BFF002801D0FEF7D5FE01B000BDC046B5
:106C7000D0100020004401405FEA0000FFF900004E
:106C800000B581B00A4800900A4901600A49416094
:106C900000218160094AC26001614161816106F0A1
:106CA0001BFF002801D0FEF7B5FE01B000BDC046B5
:106CB0008410002000480140FFF900000F27000069
:106CC00000B58DB00C900C980068012189078842AE
:106CD00009D14948026801210A430260006808405E
:106CE0000B900B9879E00C9800683D49884212D1CE
:106CF0004148026810210A430260006808400A9077
:106D00000A98112005900321002207F0BBFE059888
:106D100006F0C5FD61E00C9800683249884212D146
:106D20003548026820210A43026000680840099043
:106D30000998122004900321002207F0A3FE049872
:106D400006F0ADFD49E00C9800682749884213D150
:106D5000284802680121C9030A430260006808400C
:106D600008900898132003900321002207F08AFE60
:106D7000039806F094FD30E00C9800681B498842A7
:106D800013D11C480268012149040A4302600068CB
:106D9000084007900798152002900321002207F071
:106DA00071FE029806F07BFD17E00C980068104910
:106DB000884212D10F480268012189040A43026007
:106DC00000680840069006981620019003210022D2
:106DD00007F058FE019806F062FD0DB000BDC046F8
:106DE000001000400014004000200040004401401A
:0C6DF00000480140401002403C100240EE
:106DFC0000B583B01B4801901B490160E121490299
:106E0C00416001210A03826000230293C36089025E
:106E1C0001610C2141618361C3610362436283623E
:106E2C0019461A4605F0AAFC002801D0FEF7ECFD25
:106E3C000C48002107F06DF9002801D0FEF7E4FDA5
:106E4C000848002107F0A6F9002801D0FEF7DCFD68
:106E5C00044807F093FF002801D0FEF7D5FD03B0DE
:0C6E6C0000BDC046F40D002000380140BD
:106E780030B59BB01A900020199018901790169072
:106E8800159008A8342106F075F81A980068254965
:106E9800884245D1012008900220099008A803F0F3
:106EA80061FF002801D0FEF7B1FD1F4802680121EB
:106EB80089030A43026000680840079007981B4846
:106EC800026801210A43026000680840069006989B
:106ED800092040021590022416940020049017906F
:106EE800189001200190199005200007029015A91B
:106EF800039103F029F8019A02980399049B9502DB
:106F08001595169417921893199203F01DF8049A80
:106F18001B200590032107F0B1FD059806F0BBFC86
:106F28001BB030BD00380140401002403410024010
:106F380000B583B0029001910B490020009006F043
:106F480005F90098029906F001F90098074906F03A
:106F5800FDF80098019906F0F9F80098044906F040
:106F6800F5F803B000BDC04631F80008F0F000089D
:046F7800B1F3000869
:106F7C0000B583B0029001910B490020009006F0FF
:106F8C00E3F80098029906F0DFF80098074906F03C
:106F9C00DBF80098019906F0D7F80098044906F040
:106FAC00D3F803B000BDC04639F80008F0F0000873
:046FBC00B1F3000825
:106FC00000B583B0029001910B490020009006F0BB
:106FD000C1F80098029906F0BDF80098074906F03C
:106FE000B9F80098019906F0B5F80098044906F040
:106FF000B1F803B000BDC04641F80008F0F0000849
:04700000B1F30008E0
:1070040010B588B00B9C0A9C0790069105920493D6
:10701400069807990860079801684548086007982A
:1070240001684B20000248600798026801210803A8
:107034009060079802680020D060079A126889025D
:10704400116107990A680C215161079909688861DF
:1070540007990968C8610799096808620799096866
:107064004862079909688862059807990968486021
:107074000498002809D1079802680120810211614F
:10708400079909680003886014E0049801280AD16C
:1070940007980168032040020861079801680120ED
:1070A4000003886006E007980168002008610799DA
:1070B400096888600A98012804D1079801680020AB
:1070C400C86004E00798016801204003C86007987D
:1070D400006803900B9805F099FE00220292154B6C
:1070E40007F095F905F07AFE029B0146039800919A
:1070F40019461A4600F024F8002801D0FEF788FC4F
:107104000798006807F03EFE002801D0FEF780FCD7
:107114000799086827310122120204F047FF00286A
:1071240004D005480549FFF749FFFEE708B010BD44
:107134000038014000000C4049F80008D4F500086C
:1071440010B586B0089C04900391029201930498B0
:10715400002803D105A90120087069E0049884215E
:107164004058002806D104998022002088540498AD
:10717400FFF780FE04998422242088500498016833
:107184000868012290430860049804F0F7FA012883
:1071940003D105A9012008704AE00498806A0028F8
:1071A40002D0049806F0FEFC049801688868012265
:1071B400930318438860049800688068D103884367
:1071C400039908430499096888600298400500906F
:1071D400019801040098084300900498006800682E
:1071E40015490840009908430499096808600498FF
:1071F40001684868D3051843486004980168086822
:10720400930618430860049800684069FF21090642
:10721400084008990843049909684861049801687A
:10722400086810430860049804F008FD05A9087074
:0C72340005A8007806B010BDFFFF00FCAC
:1072400010B588B0079007980068C0690690079845
:1072500000680068059007980068806804900698A8
:107260000F2108400390039800285BD004988F49B1
:10727000084205D105A8008809214901084251D0DA
:1072800006A80078C00700280DD005A84078C007E0
:10729000002808D0079800680123036207998C2210
:1072A00088581843885006A80078800700280ED513
:1072B00004A80078C007002809D0079801680220B8
:1072C000086207998C22885804231843885006A81E
:1072D0000078400700280ED504A80078C0070028D1
:1072E00009D0079801680420086207998C22885801
:1072F00002231843885006A800780007002811D5FB
:1073000005A800788006002803D40498674908423D
:1073100008D0079800680823036207998C228858D0
:107320001843885006A840780007002819D505A8FA
:10733000C0784007002804D404A8807800060028FC
:107340000FD5079802680120C1021162079A8823AD
:107350002021D150079A8423D15055490875554AA8
:10736000885406A80078800600282BD505A8007848
:107370008006002804D404A8C078C006002821D5BF
:10738000079888214058222816D149484521C9002C
:107390004058FF2810D807980068406A44494522A1
:1073A000D2008B58CB18272418558858401C885079
:1073B000404A0120885405E007980168886908223E
:1073C0001043886106A800780006002813D505A898
:1073D00000780006002804D404A88078000600285D
:1073E00009D533480290006807F002F9029923207A
:1073F00002010120885406A80078400600280FD515
:1074000005A80078400600280AD529492622002030
:107410008854079806F0B1F80799882222208850EE
:1074200007988C21405800283DD0079988222220B7
:10743000885006A800788006002814D505A8007892
:107440008006002804D404A8C078C00600280AD505
:1074500007980168886908221043886107998C227F
:10746000002088501FE006A80078000600281AD5E2
:1074700005A800780006002804D404A88078000637
:10748000002810D50A490191262200208854079827
:1074900006F073F80199079A88232220D050232000
:1074A00002010120885408B010BDC0460100001040
:0874B000100B00203102000066
:1074B80085B00490039102A9184808800020019023
:1074C80001980399884225D204980199415C029851
:1074D800484002A90880082000900098002815D08C
:1074E80002A80088C007002808D002A90888400818
:1074F800088002980A4A5040088003E002A90888D8
:10750800400808800098401E0090E6E70198401C5B
:107518000190D5E702A8008805B07047FFFF00007A
:0475280001A00000BE
:10752C0000B585B00390039827300190039845214E
:10753C00C9004058029001980078009002980428E5
:10754C0005D8039806F044F8002004901FE0019839
:10755C00029907F07DF8401C002805D1039806F02D
:10756C0037F80020049012E00098002802D1022085
:10757C0004900CE000980749C98B884202D1022084
:10758C00049004E0039806F023F80020049004987B
:08759C0005B000BD1013002032
:1075A40010B588B006900591049203A80370007882
:1075B4003549C98B88420BD003A80078002807D02E
:1075C4000698049B06210B2206F050F8079058E019
:1075D400059988780002C9784018029005990879BD
:1075E40000024979401800900098002802D00098C1
:1075F4007E2807D30698049B0322114606F036F82A
:1076040007903EE0029800994018401E892807D34D
:107614000698049B0321022206F028F8079030E024
:107624000699049A032088540498401C04900098F6
:1076340040000699049A88540498401C04900298C7
:10764400019001980299009A8918884217D20198EA
:1076540041000D4841184978069A049BD154049975
:10766400491C049101994900405C0699049A885484
:107674000498401C04900198401C0190E1E7049890
:0C7684000790079808B010BD10130020FC
:1076900010B586B0089C0490039102920193019862
:1076A0003E49C98B88420AD00198002807D0049827
:1076B000029B06210B2205F0DBFF05906BE003998E
:1076C00088780002C978401800900098892807D36C
:1076D0000498029B0621022205F0CAFF05905AE099
:1076E00008988D21890040580099405C002807D1F6
:1076F0000498029B0621022205F0BAFF05904AE099
:1077000008988D21890040580099405C02280ED1CC
:1077100008984721C90040580088002807D10498DC
:10772000029B0621022205F0A3FF059033E0039897
:10773000007900994A0019498A18507003984079D5
:10774000009A520088540499029A0620885402989C
:10775000401C02900098000A0499029A88540298EA
:10776000401C029000980499029A88540298401C88
:107770000290039800790499029A88540298401C58
:107780000290039840790499029A88540298401C08
:10779000029002980590059806B010BD10130020C5
:1077A00010B58AB00C9C0890079106920593059835
:1077B0004F49C98B88420AD00598002807D00898FD
:1077C000069B06210B2205F053FF09908DE00799D7
:1077D00088780002C9784018049007990879000257
:1077E000497940180390072001900398002802D09F
:1077F00003987C2807D30898069B1021032205F0E4
:1078000037FF099071E0049803994018401E8928B9
:1078100007D30898069B1021022205F029FF099042
:1078200063E00498029002980499039A89188842A8
:1078300034D20C988D21890040580299405C002870
:1078400003D10198801C019024E00C988D218900BF
:1078500040580299405C02280AD10C984721C9007F
:1078600040580088002803D10198801C019011E045
:1078700007980199405C02994A001D498A18507086
:10788000079A019880184078029A5200885401980B
:10789000801C01900298401C0290C4E70899069A47
:1078A000102088540698401C06900498000A0899F5
:1078B000069A88540698401C069004980899069ADF
:1078C00088540698401C06900398000A0899069A66
:1078D00088540698401C069003980899069A885484
:1078E0000698401C06900698099009980AB010BDA9
:0478F0001013002051
:0878F40000487047EE07000098
:1078FC0085B00390029101920398019940180D49AB
:10790C00884202D30120049010E0002000900098DF
:10791C000199884208D20398009A805C0299885495
:10792C000098401C0090F2E700200490049805B0E9
:08793C007047C046010002087B
:1079440000B589B002F040FA00284DD12E4A1168E2
:107954000120430299431160022104912B490978C3
:107964004908891E0691079004A803A902F064FA45
:10797400002827D12648029000200190029825492A
:1079840088421ED802990198C300234AD018D258BD
:107994004368012002F068F9002806D102980830F3
:1079A40002900198401C01900AE0174908680122DE
:1079B40052021043086002F029FA032008901FE0E5
:1079C400DCE70AE01049086801225202104308600B
:1079D40002F01CFA0220089012E00B490868012208
:1079E40052021043086002E00120089008E002F00F
:1079F4000DFA002802D00420089001E0002008902D
:107A0400089809B000BDC04600200240E075FF1F81
:0C7A140000F0010837F00108C006002057
:107A200000B583B00190644964483822FFF766FFCF
:107A3000002802D001200290BAE05F48009000992F
:107A40000A784878000280188A78C97809028A186A
:107A500001990A83C8820098017940790002401890
:107A60000199488300988179C079000240180199F2
:107A700088830098017A407A000240180199C883EF
:107A80000098817AC07A0002401801990885009810
:107A9000017B407B00024018019948870098817C57
:107AA000C07C00024018019988870098017D407DC4
:107AB000000240180199C8870098817DC07D0002AE
:107AC00040180199422288520098017E407E0002AF
:107AD00040180199442288520098817EC07E00029D
:107AE00040180199462288520098017F407F000289
:107AF00040180199482288520098817FC07F000277
:107B0000401801994A2288520098817BC07B00026C
:107B1000401801994C2288520098017C407C000258
:107B2000401801994E2288520099084620302022A0
:107B3000895C4078000241182148018000880028B3
:107B400003D001995022012088520098014630311B
:107B50003022825C4878000280188A78C97809024D
:107B60008A1801994A810881009908462C302C22F4
:107B7000895C407800024018382802D00220029028
:107B800016E0009908462E302E22895C40780002CB
:107B90004018002802D00320029009E00098242118
:107BA000405C652802D00420029001E00020029091
:107BB000029803B000BDC046C006002000F00108D6
:047BC000EE050020AE
:107BC40070B584B0029001A801705C490091029ADA
:107BD400138B1904D48A009A1470240A54701B0A53
:107BE400D370090C91700299498B009A1171090A9A
:107BF40051710299898B009A9171090AD171029984
:107C0400C98B009A1172090A51720299098D009A5E
:107C14009172090AD1720299498F009A1173090A63
:107C240051730299898F009A9174090AD174029947
:107C3400C98F009A1175090A517502994222895A0D
:107C4400009A9175090AD17502994422895A009AB9
:107C54001176090A517602994622895A009A917638
:107C6400090AD17602994822895A009A1177090A99
:107C7400517702994A22895A009A9177090AD17751
:107C840002995622895A009B1A46203220241955FB
:107C9400090A517002994C22895A009A9173090A6F
:107CA400D17302994E22895A009A1174090A5174A7
:107CB400009B1A46283228241D5D517809024D196B
:107CC4009678D1780902891909044919491C19556A
:107CD4000B0ED3700B0C9370090A5170009B1A465B
:107CE4002C322C243821195500215170009B1A463E
:107CF4002E322E2419555170009A24236521D15413
:107D0400007800280ED002994A8910040B89009C3F
:107D140021463031302563551B0A4B70120ACA7054
:107D2400000C8870FFF70CFE002802D0012003909D
:107D340001E000200390039804B070BDC006002049
:107D440070B584B01D48029002981D492422019206
:107D540005F00AF9019A029B1946283128241D5D71
:107D64004878000245198E78C8780002801900040A
:107D74004019401C1855030ECB70030C8B70000A7D
:107D84004870029B19462C312C24382018550020A9
:107D94004870029B19462E312E24185548700299BA
:107DA40065208854FFF7CCFD002802D00220039000
:107DB40001E000200390039804B070BDC0060020C9
:047DC40010D20008D1
:107DC80000B583B00A4801A90122FFF793FD0028F6
:107DD80002D00120029008E001A80078652802D0AE
:107DE8000120029001E000200290029803B000BD3B
:047DF80024F001086A
:107DFC0000B589B001F0E4FF00284DD12E4A11687E
:107E0C000120430299431160022104912B49097806
:107E1C004908491E0691079004A803A902F008F826
:107E2C00002827D12648029000200190029825496D
:107E3C0088421ED802990198C300234AD018D25800
:107E4C004368012001F00CFF002806D1029808308D
:107E5C0002900198401C01900AE017490868012221
:107E6C0052021043086001F0CDFF032008901FE080
:107E7C00DCE70AE01049086801225202104308604E
:107E8C0001F0C0FF0220089012E00B4908680122A3
:107E9C0052021043086002E00120089008E001F053
:107EAC00B1FF002802D00420089001E000200890C7
:107EBC00089809B000BDC04600200240E075FF1FC5
:0C7ECC0000F8010811F80108F806002079
:107ED80000B583B0154801900199002000904870C2
:107EE80008700199C87088700199487108710199E2
:107EF800C87188710199487208720199C8728872AC
:107F08000199487308730199C87388730199487473
:107F18000874FFF76FFF002802D00220029001E0EA
:107F280000200290029803B000BDC046F806002069
:107F380000B583B00190314931481822FFF7DAFCC7
:107F4800002802D00120029054E02C4800900098AC
:107F580001784078000240180199012212028852E3
:107F680000988178C0780002401801998122520057
:107F780088520098017940790002401801994122FD
:107F88009200885200988179C079000240180199BE
:107F98001122120188520098017A407A0002401892
:107FA80001998322520088520098817AC07A00028F
:107FB800401801992122D20088520098017B407B09
:107FC8000002401801998522520088520098817B4E
:107FD800C07B000240180199432292008852009801
:107FE800017C407C00024018019987225200885287
:107FF80000200290029803B000BDC046F806002099
:0480080000F8010873
:10800C0000B583B001902B48009001980121090222
:10801C00405A00990870000A487001988121490063
:10802C00405A00998870000AC87001984121890053
:10803C00405A00990871000A4871019811210901F0
:10804C00405A00998871000AC8710198832149002F
:10805C00405A00990872000A487201982121C900FF
:10806C00405A00998872000AC8720198852149000B
:10807C00405A00990873000A4873019843218900FB
:10808C00405A00998873000AC873019887214900E7
:10809C00405A00990874000A4874FFF7A9FE00289A
:1080AC0002D00220029001E000200290029803B05E
:0880BC0000BDC046F8060020DB
:1080C40030B581B01F4801681F4A126851400091C1
:1080D4001E4A1168009B1940C943116013681C496A
:1080E4000C68009D2C4063400B60126809680A40CC
:1080F400009911400091009A0168514001600368A1
:1081040000990B40134A1168194311600078000765
:10811400800F002803D110494B20400108600E490C
:108124000868401E086000280AD10B4964200860D2
:10813400044802680C20024008490868104308609B
:1081440001B030BD40120020100C00505812002025
:108154005412002048120020501200204412002023
:1081640081B0009005490A68009810400090009A78
:10817400086850400860009801B070474812002019
:1081840081B0009005490A68009810400090009A58
:10819400086850400860009801B0704744120020FD
:1081A40000B581B000900448016800988843FFF747
:0C81B400D7FF01B000BDC0464012002003
:1081C00000B581B06946002008700A49086801229C
:1081D000120210430860022000F00EF8002803D0BD
:1081E00069460120087001E0FEF7A4FB68460078AC
:0881F00001B000BD00200240B7
:1081F80000B583B0029001A90020087017480078E4
:10820800002824D0164800680090144801787D2082
:10821800C00004F027FE0146009804F023FE06F093
:108228003DFC00280FD10298032808D802990022A3
:10823800D04306F023FC02980A49086002E001A92D
:108248000120087002E001A90120087002E001A9DC
:108258000120087001A8007803B000BD3A0300208F
:08826800200500200C05002098
:108270000348027803490868801808607047C046C0
:088280003A0300200C1200205B
:0C828800014800687047C0460C1200203E
:1082940000B583B00290FFF7F5FF019002980090BB
:1082A4000098401C002804D0074801780098401822
:1082B4000090FFF7E7FF0199401A0099884200D225
:0C82C400F7E703B000BDC0463A030020FD
:1082D00081B000900449086802229043009A10433C
:0C82E000086001B07047C046300001404B
:1082EC000249086801229043086070473000014041
:1082FC0081B0009004490868032252029043009A0E
:0C830C001043086001B070470000014001
:1083180000B58BB0099008A9002008700790069056
:1083280004900998002803D10AA90120087093E154
:1083380009983C21405C0128FFD109980069002870
:1083480005D009980069012149058842FFD109989B
:10835800806D002808D10998FBF72CF809990020AE
:10836800C8650999542288540998006806F0FCF9F0
:10837800002812D10998006800F082F9B84800680E
:10838800B84904F06FFD4000801C04900498002850
:1083980003D00498401E0490F8E70998006806F096
:1083A800E3F900280BD10999886D102210438865DC
:1083B800099AD16D01200143D16508A9087009986F
:1083C800006805F06DF905900998806DC0060028D1
:1083D80000D536E10598002800D032E10998806D73
:1083E80002210843012109028843099988650998EF
:1083F800006806F0C3F900284ED109980068C068E3
:108408001821884309998A6810430968C86009983F
:108418004168032292071140C06C01430698084343
:10842800069009983C21405C01280FD109994868B9
:108438000322920710400A6C10434A6C1043896C5F
:1084480008430699084301210843069009980068E3
:10845800006985490840069908430999096808612F
:108468000998406803218907884215D0099840680F
:108478000121890788420FD0099840680121C9075E
:10848800884209D0794908680F2293049843099AC9
:1084980052681A40801808600998017E8903427E54
:1084A800D2031143827E52031143026B531E9A4139
:1084B80012038918C26811430291C07C0006002883
:1084C80006D5099800690121C9078843019002E08F
:1084D80001204005019002990198014309982C2236
:1084E800805C4000014307980843079009982021C1
:1084F800405C012813D10998807E002805D107988F
:10850800012109040843079009E00999886D202290
:10851800104388650999C86D01221043C8650998F8
:10852800406A002809D00998416A0722920111403F
:10853800806A014307980843079009980068C06853
:108548004B4908400799084309990968C860099880
:10855800006800694749084006990843099909686D
:108568000861099908684A6B002105F0A2F8099981
:1085780008688A6B404905F09CF80998006900284A
:1085880007D109980168886A0F22D243104388628C
:1085980033E0099800690121490588422DD100205E
:1085A8000390039807280DD80998006E039989004D
:1085B800C8400F2108400F2800D103E00398401C51
:1085C8000390EEE70398012807D109980168886AA3
:1085D8000F22D243104388620FE009980068806A2E
:1085E8000999C8698000021F1C2002400F20C0435F
:1085F80090400A6E10430968886209980068C0684C
:108608001E490840079988420BD109990020C8657E
:108618000998806D012108430221884309998865DA
:108628000EE00998806D10210843022188430999BA
:108638008865099AD16D01200143D16508A90870A0
:1086480007E00999886D10221043886508A9012060
:10865800087008980AA908700AA800780BB000BD2D
:1086680020050020400D030002FCFF1F08270140E1
:108678001902FEFF02FCFFDF04FFFF07E7FF3F834D
:1086880081B00090009880680121090708430349D8
:1086980008400099886001B07047C046E8FFFF7F36
:1086A80000B585B00390002001900398006806F09B
:1086B80065F800285BD10398006880682F49084254
:1086C8000CD00399886D102210438865039AD16DE8
:1086D80001200143D16504A908704BE003980068A4
:1086E80000F01AFE264805F0ABF8000200280DD568
:1086F80024480068244904F0B5FB401C0190019807
:10870800002803D00198401E0190F8E70398407EA6
:1087180001282CD0FFF7B4FD029003980068006888
:10872800C007002823D10398006806F027F800281E
:1087380003D10398006800F0EFFDFFF7A1FD02994F
:10874800401A032812D3039800680068C00700285D
:108758000CD10399886D102210438865039AD16D56
:1087680001200143D16504A9087003E0D5E704A9F5
:108778000020087004A8007805B000BD170000802C
:0C8788000827014020050020400D0300E0
:1087940081B000900098806803490840001D00994A
:0C87A400886001B07047C046E8FFFF7F0E
:1087B00000B585B00390029101920398006804F01F
:1087C00073FF002860D103985421405C012803D135
:1087D00004A9022008705DE0039954220120885406
:1087E00003980068C068C00700280FD1039800688C
:1087F00005F0C8FF002803D00398006800F056F881
:1088000003980168C86801221043C8600398FFF705
:108810004BFF0146684601700078002833D1039869
:10882000806D0121090208431C49084003998865AD
:1088300003990020C8650398016D1948C862039820
:10884000016D184808630398016D17484863039841
:1088500001681C2008600399542200208854039862
:10886000016848681022104348600399086D096840
:108870004031029A019B05F0A1F8694608700398FF
:108880000068FFF787FF02E0694602200870009841
:1088900004A9087004A8007805B000BDFEF1FFFF30
:0C88A00045E80008DBD70008F1D700080D
:1088AC0081B000900098806803490840801C0099B2
:0C88BC00886001B07047C046E8FFFF7FF5
:1088C80000B59DB01B901A9119A900200870179047
:1088D8001B9800690121C907884204D01B980069C8
:1088E800E649884200D1FFE71B985421405C0128E3
:1088F80003D11CA902200870BCE11B995422012055
:1089080088541B98006804F0CBFE002800D0A2E130
:108918001A984068022800D15BE11B980069012180
:10892800C907884204D01B980069D449884206D1F7
:108938001B9800681A99096800F0AEF9F1E01B98D5
:10894800016E1A9843681F2213400F229A409143E0
:10895800169100684003002807D11A9800681F2163
:1089680089060840800E1590C2E01A980078C00762
:10897800002802D000201490B8E01A9800788007E8
:10898800002802D501201390AEE01A98007840071D
:10899800002802D502201290A4E01A980078000757
:1089A800002802D5032011909AE01A980078C00692
:1089B800002802D50420109090E01A9800788006CC
:1089C800002802D505200F9086E01A980078400606
:1089D800002802D506200E907CE01A980078000640
:1089E800002802D507200D9072E01A984078C00739
:1089F800002802D008200C9068E01A984078800778
:108A0800002802D509200B905EE01A9840784007AC
:108A1800002802D50A200A9054E01A9840780007E6
:108A2800002802D50B2009904AE01A984078C00621
:108A3800002802D50C20089040E01A98407880065B
:108A4800002802D50D20079036E01A984078400695
:108A5800002802D50E2006902CE01A9840780006CF
:108A6800002802D50F20059022E01A988078C007C8
:108A7800002802D01020049018E01A988078800707
:108A8800002802D5112003900EE01A9801680120F1
:108A9800820411401220002301939142029001D0D8
:108AA8000198029002980390039804900498059006
:108AB80005980690069807900798089008980990D6
:108AC80009980A900A980B900B980C900C980D90A6
:108AD8000D980E900E980F900F9810901098119076
:108AE8001198129012981390139814901498159046
:108AF800169815991A9A52681F231A4091400843EC
:108B08001B9908661A9840688008401C1B99C96917
:108B1800884206D81B9800681A9A5168126804F0AF
:108B280078FE1B9800681A9A1168926800F0C2F8DB
:108B38001A98C078000600284AD5514804F080FEEB
:108B480018901A9800684F4988421DD118A8807853
:108B58000006002818D418990120C0050143484888
:108B680005F02AFF4A4800684A4904F07BF90146A3
:108B78000C2048430C3017901798002803D01798FA
:108B8800401E1790F8E723E01A9800683E4988428B
:108B98000CD118A8C078C007002807D1189901205F
:108BA80000060143364805F007FF11E01A980068EF
:108BB800364988420CD118A880784006002807D486
:108BC80018990120800501432D4805F0F5FEFFE7BF
:108BD80040E01B9800690121C907884204D01B980E
:108BE80000692649884205D11B9800681A990968C6
:108BF80000F074F81A98C078000600282AD5204892
:108C080004F01EFE18901A9800681E49884207D181
:108C180018990120C0058143194805F0CDFE19E0D7
:108C28001A9800681849884207D118990120000647
:108C38008143134805F0C0FE0CE01A9800681349F8
:108C4800884207D118990120800581430C4805F016
:108C5800B3FEFFE707E01B99886D20221043886563
:108C680019A9012008701B995422002088541998CA
:108C78001CA908701CA800781DB000BD0400008065
:108C880008270140001000B0004000B8002000B4E0
:088C980020050020400D03003F
:108CA00082B001900091009A034802400199886ABD
:0C8CB0001043886202B07047FFFF07000D
:108CBC0083B00290019100920298406901990A02D6
:108CCC00904300991140034A1140084302994861AE
:088CDC0003B0704700FFFF0721
:108CE40082B0019000910098C24304480243019964
:108CF400886A1040886202B07047C0460000F8FFDE
:108D040000B5B3B0319030912FA90020087030988D
:108D14004068032189058842FFD131983C21405C99
:108D2400012800D1FFE731985421405C012803D188
:108D340032A9022008708DE231995422012088540E
:108D44003198006804F0AEFC002800D054E230985A
:108D54000068E64988423ED1309840682C90012151
:108D6400C905884212D02C9803218905884214D160
:108D740031980068309989687F22D2049143032294
:108D840092058A18D94900F06FFA0CE0319800680E
:108D9400D649D74A00F068FA05E031980068D3490B
:108DA400002200F061FA3199886D01221204904387
:108DB40088653198006804F04EFD3098007B0128E6
:108DC40004D13198006804F04DFD03E03198006847
:108DD40004F051FD10E2309840682B900121C90540
:108DE400884200D1C5E12B9803218905884200D02F
:108DF400C7E130980068BF49884200D0D9E0309874
:108E040080684003002807D1309880681F218906B4
:108E14000840800E2A90C2E03098007AC0070028EB
:108E240002D000202990B8E03098007A800700280A
:108E340002D501202890AEE03098007A400700283F
:108E440002D502202790A4E03098007A0007002879
:108E540002D5032026909AE03098007AC0060028B4
:108E640002D50420259090E03098007A80060028EE
:108E740002D50520249086E03098007A4006002828
:108E840002D5062023907CE03098007A0006002862
:108E940002D50720229072E03098407AC00700285B
:108EA40002D00820219068E03098407A800700289A
:108EB40002D5092020905EE03098407A40070028CF
:108EC40002D50A201F9054E03098407A0007002809
:108ED40002D50B201E904AE03098407AC006002844
:108EE40002D50C201D9040E03098407A800600287E
:108EF40002D50D201C9036E03098407A40060028B8
:108F040002D50E201B902CE03098407A00060028F1
:108F140002D50F201A9022E03098807AC0070028EA
:108F240002D01020199018E03098807A8007002829
:108F340002D5112018900EE0309881680120820437
:108F440011401220002316939142179001D01698D5
:108F54001790179818901898199019981A901A98A9
:108F64001B901B981C901C981D901D981E901E9879
:108F74001F901F9820902098219021982290229849
:108F84002390239824902498259025982690269819
:108F94002790279828902898299029982A902A98E9
:108FA4000123834031980168A022885818438850CF
:108FB400DEE0309880684003002807D1309880684C
:108FC4001F2189060840800E1590C8E03098007A69
:108FD400C007002802D000201490BEE03098007A28
:108FE4008007002802D501201390B4E03098007A5D
:108FF4004007002802D502201290AAE03098007A97
:109004000007002802D503201190A0E03098007AD0
:10901400C006002802D50420109096E03098007A0B
:109024008006002802D505200F908CE03098007A45
:109034004006002802D506200E9082E03098007A7F
:109044000006002802D507200D9078E03098407A79
:10905400C007002802D008200C906EE03098407AB7
:109064008007002802D509200B9064E03098407AEC
:109074004007002802D50A200A905AE03098407A26
:109084000007002802D50B20099050E03098407A60
:10909400C006002802D50C20089046E03098407A9B
:1090A4008006002802D50D2007903CE03098407AD5
:1090B4004006002802D50E20069032E03098407A0F
:1090C4000006002802D50F20059028E03098807A09
:1090D400C007002802D0102004901EE03098807A47
:1090E4008007002808D51120039014E00000C07CFC
:1090F400FFFF8700FFFF170030988168012082047A
:1091040011401220002301939142029001D0019852
:10911400029002980390039804900498059005988F
:10912400069006980790079808900898099009985F
:109134000A900A980B900B980C900C980D900D982F
:109144000E900E980F900F981090109811901198FF
:1091540012901298139013981490149815901598CF
:109164000123834031980168A42288581843885009
:109174000EE03198006830990968394A00F074F8B3
:1091840006E03198006830990968002200F06CF814
:10919400309800683349884217D13199886D01228B
:1091A4005204904388653198006805F015FC3098A6
:1091B400007B012804D13198006805F015FC03E018
:1091C4003198006805F01AFC16E03199886D012287
:1091D4009204904388653198006805F019FC309832
:1091E400007B012804D13198006805F019FC03E0E4
:1091F4003198006805F01EFC3098006817498842D1
:1092040013D13098006931990968C968182211404E
:10921400890888402E903098406931990968C96856
:109224001140890888402D9005E0309800692E90FF
:10923400309840692D9031980068309909682E9AC9
:109244002D9B00F039F831995422002088542F982E
:1092540032A9087032A8007833B000BD0000C07C89
:08926400FFFF8700FFFF170068
:10926C0084B003900291019202980F49884203D175
:10927C0003980C30009008E00398029901225205E3
:10928C001140C90C4018A030009000980068029A58
:10929C00D143064B194308400199114008430099EA
:1092AC00086004B07047C0460000C07C00003883E2
:1092BC0085B004900391029201930498039A0321C0
:1092CC000B0511461940090D01235B051A40520D7F
:1092DC0089188900401820300090009800680549D2
:1092EC00084002990904019A114308430099086047
:0892FC0005B0704700F000F01E
:1093040081B00090009880680349084010300099AB
:0C931400886001B07047C046E8FFFF7F92
:1093200081B000900098806803490840401C009973
:0C933000886001B07047C046E8FFFF7F76
:10933C0000B585B003900020019003985421405C47
:10934C00012803D104A90220087061E0039954227A
:10935C0001208854039805F017FA02A908700398A5
:10936C00006805F06DFB002846D10398806D022142
:10937C000843012211028843039988650398006809
:10938C00C06803231840009003980168C86898438C
:10939C00C860039801688868D207104388600398F6
:1093AC00006805F055FB002817D00198401C01906F
:1093BC000198194988420FD30398806D10210843F6
:1093CC00022188430399886503995422002088540C
:1093DC0004A9012008701BE0E1E7009A03980168DA
:1093EC00C8681043C8600398806D012108430221AE
:1093FC0088430399886504E00399886D1022104313
:10940C0088650399542200208854029804A9087096
:0C941C0004A8007805B000BD00F20200BA
:1094280070B582B0024601A8027000910021405632
:10943800002815D4002401A908570322D343184053
:10944800164A805809578C07E50EFF24AC40A04304
:10945800009CA401E4B2AC4020431940885019E0B4
:1094680001A908780F24204008380322D343184064
:10947800094A8058002549578D07EE0EFF25B5404B
:10948800A843009DAD01EDB2B540284321400839FD
:109498001940885002B070BD1CED00E000E400E007
:1094A80081B001466846017000214056002807D463
:1094B800684601781F200140012088400149086062
:0894C80001B0704700E100E073
:1094D00081B00146684601700021405600280BD437
:1094E000684601781F200140012088400349086038
:1094F000BFF34F8FBFF36F8F01B0704780E100E083
:10950000BFF34F8F034904480860BFF34F8F00BF7C
:0C951000FDE7C0460CED00E00400FA0589
:10951C0000B583B001900198401E000E002802D0C7
:10952C000120029010E00198401E094908600020BB
:10953C000090C0430321FFF771FF009805490860B4
:10954C00054A072111600290029803B000BDC04685
:0C955C0014E000E018E000E010E000E087
:1095680000B583B001900198002803D102A9012019
:10957800087050E00198407F002805D1019900202B
:1095880008770198F9F7A8FF019902204877019810
:10959800007900280CD10198016821484861019898
:1095A80000688068182188430199096888600AE082
:1095B80001988168C26803F045FE002803D002A91B
:1095C8000120087027E001984079002805D101980A
:1095D80001680020C043086103E00199086909682F
:1095E80008610198006880686021884301994A6988
:1095F8001043096888600198006880688021884362
:1096080001998A691043096888600199012048779F
:1096180002A90020087002A8007803B000BDC04667
:04962800B71DC104A5
:10962C0010B588B006900591049200200190059821
:10963C0000690128FFD1059800680428FFD106981D
:10964C004079012803D107A902200870DFE00699B0
:10965C0001204871069902200871059800680428B9
:10966C0065D10498002823D1FEF708FE01900698D6
:10967C000068406B0004002811D5FEF7FFFD01992E
:10968C00401A02280AD30699086908221043086177
:10969C0006990320087107A90870B8E0E7E70120D4
:1096AC00FEF7F2FD059880690699096808641FE0C9
:1096BC0006980068406BC00F002811D0FEF7DEFD45
:1096CC000199401A02280AD3069908690822104306
:1096DC00086106990320087107A9087097E0E7E76D
:1096EC000120FEF7D1FD0598806906990968486448
:1096FC0006980068806C049B10210B40464A9A40E7
:10970C009043059AD2699A401043069A1268906465
:10971C0006980068C06C049A0A40FF219140884367
:10972C000599096A9140084306990968C864059827
:10973C000069012819D106980068806B0390049881
:10974C00102210401F2181400398884303900598F4
:10975C004069029002990498104081400398084394
:10976C000390039806990968886306980068C06B93
:10977C0003900498102210400721814003988843DD
:10978C000390059908688B681843C96808430290D0
:10979C000299049810408140039808430390039861
:1097AC0006990968C86304991140012084038C4010
:1097BC0006990B681968A14319600699096809682C
:1097CC00039104991140154B8B40039999430391D4
:1097DC00059949680291029B049911408B400399A9
:1097EC00194303910399069B1B6819600499114056
:1097FC00C0238B4006990A68116899431160069939
:10980C00087106990020487107A90020087007A864
:10981C00007808B010BDC046FF030000FE0F00002A
:10982C0000B585B003900398002803D104A901204A
:10983C00087066E0039801900068344940181421C0
:10984C0003F00EFB01998000086403992522022085
:10985C0088540398016808682D4A104008600398E2
:10986C0002908268C1680A4301690A4341690A434C
:10987C0081690A43C1690A43016A0A43016808689D
:10988C0010430860039800F045F8039880680121A4
:10989C008903884202D103990020486003994868E3
:1098AC003F221040496C08600399C86C896C486071
:1098BC000398406800280FD00398406804280BD800
:1098CC00039800F049F80398016D00200860039993
:1098DC00886D496D486006E003990020086503997E
:1098EC0048650399886503990020C863039925226C
:1098FC0001208854039924220020885404A90020B4
:10990C00087004A8007805B000BDC046F8FFFDBF84
:04991C000F80FFFFBA
:1099200000B583B002900299086C032290430B4A61
:1099300080184864029800780838142103F096FAD9
:10994000019002990648886401991F200140012076
:1099500088400299C86403B000BDC04600080240B8
:049960008008024039
:1099640082B00190019840683F210840009000981F
:10997400800008494018019908650199064848651E
:109984000098411E03200140012088400199886508
:0C99940002B07047FC080240400902408D
:1099A00084B003900291019200930399C86C896C72
:1099B00048600398006D002803D00399886D496DB5
:1099C00048600398006C1C210840012282400F4926
:1099D0000868104308600098039909684860039874
:1099E0008068102808D10198039909688860029856
:1099F00003990968C86007E00298039909688860BC
:109A0000019803990968C86004B0704704000240D7
:109A100082B000900098002803D101A901200870AD
:109A200048E000982521405C02280AD000990420D3
:109A3000C863009924220020885401A901200870DD
:109A400038E00098016808680E229043086000988A
:109A5000416C08680122130298430860009801686D
:109A60000868904308600098006C1C210840824000
:109A700012490868104308600099C86C896C4860F6
:109A80000098006D00280AD00098016D0868012236
:109A90001202904308600099886D496D48600099F2
:109AA000252201208854009924220020885401A9ED
:109AB0000020087001A8007802B07047040002403E
:109AC00000B587B0059004A8017003920598252180
:109AD000405C02280AD005990420C8630599242215
:109AE0000020885406A901200870B7E00598006896
:109AF00000688006002806D5059A01200102D1637E
:109B000006A90870AAE004A80078002807D10598E3
:109B1000016C1C20014002208840029006E005985C
:109B2000016C1C200140042088400290FEF7ACFB31
:109B300001904C480068029908423FD149480068AA
:109B40000599096C1C221140C8400007002817D550
:109B50000598016C1C200140012003468B40424ABD
:109B60001168194311600599C86305992522885425
:109B7000059924220020885406A9012008706DE070
:109B80000398401C002818D0FEF77EFB0199401A6C
:109B90000399884202D8039800280ED10599202005
:109BA000C8630599252201208854059924220020A4
:109BB000885406A90120087050E0BAE70598006DA6
:109BC000002816D00598406D00680599896D0842F7
:109BD0000FD00598016D0868012213021843086030
:109BE0000599886D496D48600599C86B92021043CC
:109BF000C8630598806C00680599C96C084209D053
:109C00000599C86C896C48600599C86B012252029D
:109C10001043C86304A80078002812D10598006C8E
:109C20001C210840022282400F4908681043086046
:109C30000599242200208854059925220120885462
:109C400009E00598006C1C21084004228240064966
:109C500008681043086006A90020087006A800786C
:0C9C600007B000BD0000024004000240FC
:109C6C0010B588B006900591039302921C480078B9
:109C7C00012803D107A9022008702DE01849012002
:109C8C0008701749002048607D20C00000F034F8AF
:109C9C00014601A801700078002817D10698012808
:109CAC0005D10598039B029A00F074F803E005981F
:109CBC00029900F019F87D20C00000F01DF801A9F0
:109CCC000870069A07490868904308600449002008
:109CDC000870019807A9087007A8007808B010BD93
:109CEC008C1100201420024008B4024B9C4608BC86
:089CFC006047C04699040020F6
:109D040000B585B00390FEF7BDFA039940180190A1
:109D14000120000402901D4800680299084209D0FD
:109D2400FEF7B0FA0199884203D304A9032008700E
:109D340028E0F0E715490868154A104002901548D4
:109D440008600298002806D002981349486004A9C4
:109D54000120087016E0FEF795FA03994018019067
:109D64000A4800684003002809D5FEF78BFA0199D8
:109D7400884203D304A90320087003E0F0E704A990
:109D84000020087004A8007805B000BD102002402F
:0C9D9400FAC30000FBC300008C1100208B
:109DA00084B0039001930092074908680122104390
:109DB0000860009803990860BFF36F8F01980399BA
:0C9DC000486004B07047C0461420024008
:109DCC0081B06946002008700A480068C00F00285E
:109DDC000CD0094909480860094808600548006822
:109DEC00C00F002802D06946012008706846007830
:109DFC0001B070471420024008200240230167453F
:049E0C00AB89EFCD62
:109E100081B068460122027007480168D2071143E9
:109E200001600068C00F002802D069460020087059
:0C9E30006846007801B070471420024022
:109E3C0000B585B0039002912E480078012803D11B
:109E4C0004A90220087051E02A4901200870294910
:109E5C00002048607D20C000FFF74EFF014601A89E
:109E6C000170007800283BD10399042048600398C6
:109E7C00006804280AD10398406800F03FF87D2060
:109E8C00C000FFF739FF01A9087029E002990020F2
:109E9C00C04308600398806800900098039A91680A
:109EAC00D2688918884216D203984068009900F04D
:109EBC0033F87D20C000FFF71FFF014601A8017099
:109ECC000078002803D000980299086003E00098FD
:109EDC00401C0090E1E708490868022290430860A2
:109EEC00044900200870019804A9087004A800789F
:0C9EFC0005B000BD8C11002014200240B5
:109F080081B00090009804490A68104301221204A5
:0C9F18001043086001B0704714200240A4
:109F240083B002900191074908683F22D200904310
:109F34000090009A0198C0001043034A104308603F
:0C9F440003B0704714200240020001002E
:109F50008AB0099008910020079008980068079936
:109F6000C840002800D130E108980068079A012114
:109F70009140084006900698002800D121E10898F9
:109F8000406803210840012805D008984068032153
:109F9000084002282AD10998806805900798400057
:109FA000032181400598884305900898C168079867
:109FB00040008140059808430590059809998860FC
:109FC00009984068059007980121814005988843C9
:109FD00005900898406810210840010907988140C1
:109FE00005980843059005980999486008984068C5
:109FF00003210840032814D00998C06805900798E9
:10A0000040000321814005988843059008988168A5
:10A0100007984000814005980843059005980999E4
:10A02000C860089840680321084002281ED109989A
:10A030000799C90889004018006A059007984007E9
:10A04000C00E0F218140059888430590089801694A
:10A0500007984007C00E8140059808430590059871
:10A060000999079AD208920089180862099800682D
:10A07000059007984100032002468A4005999143C4
:10A08000059108994968014007984000814005986A
:10A090000843059005980999086008988079800719
:10A0A000002800D18DE00798032188434849405893
:10A0B000059007988007C00E0F21814005988843BE
:10A0C0000590099805210907884202D100200490D3
:10A0D0001DE009983F49884202D10120039014E015
:10A0E00009983D49884202D1022002900BE009996B
:10A0F0003A4A0320052300939142019001D0009831
:10A10000019001980290029803900398049004999A
:10A1100007988007C00E8140059808430590059870
:10A120000799032291432A4A88502D4800680590D8
:10A13000069905988843059008988079C0070028FB
:10A1400003D00699059808430590059824490860AE
:10A15000244800680590069905988843059008985A
:10A1600080798007002803D5069905980843059053
:10A1700005981C4908601C480068059006990598D8
:10A180008843059008988079C006002803D5069971
:10A19000059808430590059813490860134800681E
:10A1A000059006990598884305900898807980065F
:10A1B000002803D5069905980843059005980B4992
:10A1C00008600798401C0790C7E60AB07047C04671
:10A1D000601802400004005000080050000C0050BD
:10A1E00080180240841802400018024004180240FF
:10A1F0008BB00A9009910020089009980899C840EE
:10A20000002800D198E00998089A0121914008405F
:10A2100007900798002800D18AE008980321884316
:10A2200046494058069008988007C00E0F2181408B
:10A23000069808400690069805900A980521090797
:10A24000884202D1002004901DE00A983C498842CF
:10A2500002D10120039014E00A983A49884202D1C1
:10A26000022002900BE00A99374A0320052300934D
:10A270009142019001D000980190019802900298BB
:10A2800003900398049005980499089A9207D20EB7
:10A290009140884221D1079A2C4908689043086070
:10A2A000079A2B49086890430860079A294908686B
:10A2B00090430860079A2849086890430860089806
:10A2C0008007C10E0F2088400690069B0899032046
:10A2D00081431A4A885898438850089840000322BE
:10A2E000134683400A99086818430860089948078C
:10A2F000C00E0F2383400A98C90889004118086AD4
:10A300009843086208984000134683400A99886879
:10A31000984388600898012383400A9948689843C5
:10A3200048600898400082400A99C8689043C86015
:10A330000898401C089060E70BB070476018024016
:10A340000004005000080050000C0050801802402B
:0CA350008418024000180240041802406B
:10A35C0000B583B00190174908680322520290435C
:10A36C00019A10430860019801214902884219D1D1
:10A37C001148016806204843104902F071FD401C49
:10A38C0000900F480068400500280BD50098002865
:10A39C0003D00098401E009003E002A9032008702F
:10A3AC0003E0EEE702A90020087002A8007803B0D1
:10A3BC0000BDC046007000402005002040420F0048
:04A3CC0014700040C9
:10A3D00010B588B006900698002803D107A901207F
:10A3E0000870CEE206980078C007002873D0FA48BB
:10A3F0000068382108400490F848006803210840AC
:10A4000003900498102802D10398032802D00498DE
:10A4100008280DD1F24800688003002807D5069867
:10A420004068002803D107A901200870A9E252E082
:10A430000698406801210904884206D1E849086865
:10A4400001221204104308601AE0069840680521B2
:10A45000090488420AD1E24908680122930418439A
:10A460000860086812041043086009E0DC490868C5
:10A47000012213049843086008689204904308601E
:10A4800006984068002813D0FDF7FEFE0590D448DA
:10A490000068800300280AD4FDF7F6FE0599401AEB
:10A4A000652803D307A9032008706AE2EFE712E0EA
:10A4B000FDF7EAFE0590CA480068800300280AD527
:10A4C000FDF7E2FE0599401A652803D307A903208A
:10A4D000087056E2EFE7069800788007002800D45D
:10A4E00090E0BD480068382108400490BB480068EF
:10A4F0000321084003900498102802D103980228F1
:10A5000002D00498002834D1B548006840050028DE
:10A5100007D50698C068002803D107A90120087054
:10A520002FE2B04908687F2212029043069A5269CE
:10A53000120210430860049800280FD1A84802684E
:10A540000721C9028A43069B1B691A4302600068FF
:10A550000840C10AA448C840A4490860A44800684B
:10A56000FDF74AFE002803D007A90120087008E281
:10A5700048E00698C06800282BD09949086807224F
:10A58000D2029043069A12691043086008680122BB
:10A59000120210430860FDF777FE0590FD48006841
:10A5A000400500280AD4FDF76FFE0599401A0328DC
:10A5B00003D307A903200870E3E1EFE7F649086831
:10A5C0007F2212029043069A5269120210430860D9
:10A5D00018E0F04908680122120290430860FDF774
:10A5E00053FE0590EB480068400500280AD5FDF7AA
:10A5F0004BFE0599401A032803D307A903200870CE
:10A60000BFE1EFE7069800780007002848D5DF484B
:10A6100000683821084018280DD1E04800688007FC
:10A62000002807D506988069002803D107A90120D2
:10A630000870A6E134E006988069002818D0D74950
:10A640000868012210430860FDF71EFE0590D348FC
:10A650000068800700280AD4FDF716FE0599401A05
:10A66000032803D307A9032008708AE1EFE717E066
:10A67000CA490868012290430860FDF705FE05906D
:10A68000C6480068800700280AD5FDF7FDFD05993A
:10A69000401A032803D307A90320087071E1EFE7EC
:10A6A000069800784007002800D4ADE002A90020F9
:10A6B0000870B64800683821084020280DD1BA48F3
:10A6C00000688007002807D506988068002803D115
:10A6D00007A90120087054E196E0B1480068C00065
:10A6E00000280CD4AE480268012109070A43026021
:10A6F000006808400190019802A901200870A9484B
:10A700000068C005002818D4A64908680122120272
:10A7100010430860FDF7B8FD0590A2480068C00529
:10A7200000280AD4FDF7B0FD0599401A032803D389
:10A7300007A90320087024E1EFE706988068012844
:10A7400005D19949086801221043086016E006986F
:10A750008068052809D194490868042210430860DC
:10A76000086801221043086008E08F490868012248
:10A770009043086008680422904308600698806847
:10A78000002814D0FDF780FD0590874800688007F9
:10A7900000280BD4FDF778FD0599401A83498842BB
:10A7A00003D307A903200870EBE0EEE722E0FDF7F2
:10A7B0006BFD05907C480068800700281AD5FDF7DE
:10A7C00063FD0599401A7949884203D307A90320FC
:10A7D0000870D6E0EEE7C046081002400C100240B8
:10A7E00000100240041002400024F4002005002064
:10A7F0000C05002002A80078012805D168490868E6
:10A8000001221207904308600698C069002800D111
:10A81000B4E05E48006838210840102870D00698DF
:10A82000C069022849D15B49086801221206904399
:10A830000860FDF729FD0590564800688001002852
:10A840000AD5FDF721FD0599401A032803D307A96E
:10A850000320087095E0EFE74D490868554A10401D
:10A86000069B1A6A5C6A22439C6A24022243DC6AC1
:10A8700022431C6B22435B6B1A4310430860454B19
:10A880001868012214062043186008681207104354
:10A890000860FDF7F9FC05903E480068800100283B
:10A8A0000AD4FDF7F1FC0599401A032803D307A940
:10A8B0000320087065E0EFE721E0364908680122CF
:10A8C00012069043086032490868032290430860EA
:10A8D0000868374A10400860FDF7D6FC05902D48FF
:10A8E0000068800100280AD5FDF7CEFC0599401AC2
:10A8F000032803D307A90320087042E0EFE73DE0F7
:10A900000698C069012803D107A90120087038E022
:10A910001F48006803900398032108400699096ABC
:10A92000884227D10398702108400699496A8842D5
:10A9300020D103987F21090208400699896A0902FB
:10A94000884217D103981F21490408400699C96A13
:10A9500088420FD103980721490608400699096BE0
:10A96000884207D103980721490708400699496B97
:10A97000884203D007A90120087002E007A900203F
:10A98000087007A8007808B010BDC0460810024043
:10A990000C100240001002400410024060100240FF
:10A9A0003C100240007000405C100240891300001F
:08A9B000FFFFFEEE8C80C111D7
:10A9B80000B585B0039002910398002803D104A93B
:10A9C80001200870E9E002987649096807221140D9
:10A9D80088421CD97349086807229043029A104399
:10A9E8000860FDF74DFC01906E480068072108409B
:10A9F800029988420BD0FDF743FC0199401A71492E
:10AA0800884203D304A903200870C6E0ECE7039842
:10AA180000788007002813D503980078400700289D
:10AA280005D56149086807221203104308605E498A
:10AA380008680F2212029043039A92681043086034
:10AA480003980078C007002860D003984068012860
:10AA580009D1584800688003002803D404A90120BC
:10AA680008709AE032E003984068022809D15148FA
:10AA780000688001002803D404A9012008708CE034
:10AA880024E003984068002809D14A480068400536
:10AA9800002803D404A9012008707EE016E003987A
:10AAA8004068032809D1424800688007002803D479
:10AAB80004A90120087070E008E03C48006880079D
:10AAC800002803D404A90120087066E03649086804
:10AAD80007229043039A526810430860FDF7D0FBA1
:10AAE8000190314800683821084003994968C90035
:10AAF80088420BD0FDF7C4FB0199401A31498842BE
:10AB080003D304A90320087047E0EAE7029825491F
:10AB180009680722114088421CD222490868072286
:10AB28009043029A10430860FDF7AAFB01901D4864
:10AB3800006807210840029988420BD0FDF7A0FB66
:10AB48000199401A1F49884203D304A903200870B9
:10AB580023E0ECE7039800784007002808D512495D
:10AB68000868072212039043039AD26810430860CA
:10AB780000F02AF80C4909680F22120211408A09CC
:10AB88000D4989581F221140C8400C4908600C48DB
:10AB98000068FDF72DFB04A9087004A8007805B02B
:10ABA80000BDC04600200240081002405C10024070
:10ABB80060100240001002404432000820050020C6
:08ABC8000C05002089130000B8
:10ABD00000B587B03A4800688006400F00280ED1C3
:10ABE0003B4800680721C9020840C10A012088408B
:10ABF00002900299354802F039F901905CE0304842
:10AC0000006838210840082802D12F48019053E0FD
:10AC10002B48006838210840102837D1294801689E
:10AC20000322114005910068702108400009401C72
:10AC3000039005980090022810D0009803280DD1A9
:10AC40000399214802F012F901461E4800687F224C
:10AC500012021040000A484306900CE003991B487A
:10AC600002F004F90146174800687F2212021040E2
:10AC7000000A4843069013480068400F401C0490A7
:10AC80000698049902F0F2F8019015E00C4800686B
:10AC900038210840202803D10120C00301900BE097
:10ACA0000748006838210840182803D17D20000299
:10ACB000019001E000200190019807B000BDC0465E
:10ACC000081002400C10024000127A000024F40028
:04ACD000001002402E
:0CACD400014800687047C04620050020C1
:10ACE00000B581B0FFF7F6FF009000F00DF80146C7
:10ACF0000098090B8A00034989581F221140C84057
:08AD000001B000BD843200081F
:10AD080002480068072109030840704708100240FC
:10AD1800034908680122D204104308607047C046FE
:04AD280000100240D5
:10AD2C0000B581B00C48006800900098032109021E
:10AD3C0008400A49086068464078C007002801D0DE
:10AD4C0002F0C2FE684640788007002801D502F068
:10AD5C00BCFE01B000BDC0461C10024020100240D9
:10AD6C0000B587B0069003A90020087002A90870EE
:10AD7C00069880788007002800D487E001A900207D
:10AD8C000870A6480068C00000280CD4A3480268CC
:10AD9C00012109070A4302600068084000900098EE
:10ADAC0001A9012008709E49086801221202104373
:10ADBC000860FDF763FA049099480068C005002804
:10ADCC000AD4FDF75BFA0499401A032803D303A9AC
:10ADDC000320087000E0EFE703A80078002848D1B2
:10ADEC009048006803210902084005900598002846
:10ADFC0014D005980699096B88420FD089490868C8
:10AE0C000322120290430590086801221204104399
:10AE1C0008600868904308600598086005A80078E9
:10AE2C00C007002813D0FDF729FA04907D4800686C
:10AE3C00800700280BD4FDF721FA0499401A7A49AF
:10AE4C00884203D303A90320087000E0EEE703A8AF
:10AE5C000078002809D17349086803221202904334
:10AE6C00069A126B1043086002E0039802A908705E
:10AE7C0002E0039802A9087001A80078012805D106
:10AE8C00664908680122120790430860069800780A
:10AE9C00C007002807D06549086803229043069A2A
:10AEAC00526810430860069800788007002807D580
:10AEBC005E4908680C229043069A92681043086019
:10AECC0006980078C006002808D55849086803225F
:10AEDC0092029043069AD268104308600698407814
:10AEEC008007002808D55149086803229204904332
:10AEFC00069A92691043086006984078400700282B
:10AF0C0008D54A490868032212059043069AD2696B
:10AF1C0010430860069800788006002808D543493D
:10AF2C000868032212039043069A126910430860C2
:10AF3C00069840784006002814D53C49086803223E
:10AF4C0092079043069A126A104308600698006AAA
:10AF5C0001218907884205D135490868012212046C
:10AF6C0010430860069880780007002807D52F4901
:10AF7C00086840229043069A526A1043086006986B
:10AF8C0080788006002812D5284A1068012189058E
:10AF9C008843069B9B6A184310600698806A884217
:10AFAC0005D123490868012212061043086006984F
:10AFBC0080784006002812D51C4A10680121090629
:10AFCC008843069BDB6A184310600698C06A884267
:10AFDC0005D117490868012212061043086006982B
:10AFEC0040780007002814D5104908680322920302
:10AFFC009043069A526910430860069840690121F3
:10B00C008903884205D10A490868012212041043B9
:10B01C00086002A8007807B000BDC0463C10024092
:10B02C00007000405C100240891300005410024074
:04B03C000C100240B2
:10B0400083B0029001910298006800900298334901
:10B05000884208D0029801218907884203D00298CB
:10B060002F49884208D100987021884300900198A8
:10B07000416800980843009002982849884218D0F7
:10B08000029801218907884213D0029824498842F6
:10B090000FD00298234988420BD002982249884257
:10B0A00007D002982149884203D00298204988425B
:10B0B00009D1009803210902884300900198C168D2
:10B0C00000980843009000988021884301994969BD
:10B0D00008430090009802990860019880680299DE
:10B0E000C862019800680299886202980B498842F8
:10B0F0000BD002980C49884207D002980B4988422D
:10B1000003D002980A49884203D101980069029944
:10B11000086302990120486103B07047002C014088
:10B120000004004000200040004001400044014075
:04B130000048014092
:10B1340083B0019001983D21405C012803D002A90D
:10B144000120087036E001993D22022088540198BC
:10B1540000681A4988420FD00198006801218907C4
:10B16400884209D0019800681549884204D00198A2
:10B1740000681449884214D1019800688068124913
:10B1840008400090009806280AD00098012109047C
:10B19400884205D0019801680868012210430860BC
:10B1A40005E001980168086801221043086002A9BB
:10B1B4000020087002A8007803B07047002C0140FA
:0CB1C400000400400040014007000100B2
:10B1D00083B0019001983D21405C012803D002A971
:10B1E000012008703CE001993D220220885401981A
:10B1F0000168C86801221043C860019800681A49B4
:10B2000088420FD00198006801218907884209D03F
:10B21000019800681549884204D0019800681449D3
:10B22000884214D101980068806812490840009053
:10B23000009806280AD0009801210904884205D008
:10B2400001980168086801221043086005E0019830
:10B250000168086801221043086002A900200870F4
:10B2600002A8007803B07047002C014000040040A1
:08B2700000400140070001004D
:10B2780081B0009000980168C86801229043C860B6
:10B2880000980068006A0B4908420BD100980068D2
:10B29800006A0949084205D1009801680868012236
:10B2A8009043086000993D2201208854002001B095
:0CB2B8007047C046111100004404000063
:10B2C40000B581B000900098006800690221084030
:10B2D4004008002822D000980068C0680221084075
:10B2E400400800281AD0009801680220C043086171
:10B2F4000099012008770098006880698007002879
:10B3040003D0009803F062FC05E0009803F062FCAF
:10B31400009803F063FC0099002008770098006807
:10B324000069042108408008002823D000980068A0
:10B33400C06804210840800800281BD000980168D8
:10B344000420C0430861009902200877009800682F
:10B3540080698005800F002803D0009803F036FC34
:10B3640005E0009803F036FC009803F037FC0099E0
:10B374000020087700980068006908210840C00888
:10B38400002822D000980068C06808210840C0083E
:10B3940000281AD0009801680820C0430861009969
:10B3A4000420087700980068C0698007002803D04B
:10B3B400009803F00BFC05E0009803F00BFC0098E8
:10B3C40003F00CFC009900200877009800680069DD
:10B3D400102108400009002823D000980068C068A4
:10B3E40010210840000900281BD000980168102093
:10B3F400C043086100990820087700980068C06974
:10B404008005800F002803D0009803F0DFFB05E0DF
:10B41400009803F0DFFB009803F0E0FB00990020A4
:10B424000877009800680069C00700280DD00098CC
:10B434000068C068C007002807D000980168012090
:10B44400C04308610098FBF7E5FA009800680069BA
:10B45400C0B2C00900280ED000980068C068C0B20D
:10B46400C009002807D0009801688020C043086103
:10B47400009803F011FC009800680069012109029A
:10B484000840000A00280DD000980068C068C0B2C7
:10B49400C009002806D0009801681B48086100987C
:10B4A40003F0FEFB00980068006940210840800911
:10B4B40000280FD000980068C06840210840800927
:10B4C400002807D0009801684020C0430861009814
:10B4D40003F088FB009800680069202108404009B7
:10B4E40000280FD000980068C06820210840400957
:10B4F400002807D0009801682020C0430861009804
:0CB5040003F0C6FB01B000BDFFFEFFFF1E
:10B5100000B585B00390029103983C21405C01285E
:10B5200003D104A9022008709CE003993C22012069
:10B53000885403993D22022088540398006880684B
:10B54000019001984949084001900198FF210902A2
:10B5500088430190019803990968886002980068FF
:10B56000009000286CD00098102869D000982028FE
:10B5700066D00098302863D00098402853D00098B7
:10B58000502836D00098602840D0009870280BD002
:10B59000009801210903884205D000980121490340
:10B5A000884216D053E052E003980068029B9968E5
:10B5B0005A68DB6802F0DDFA039800688068019041
:10B5C00001987721084301900198039909688860E0
:10B5D0003DE003980068029B99685A68DB6802F0B6
:10B5E000C8FA0398016888680122920310438860B2
:10B5F0002DE003980068029A5168D26803F0F8FAC7
:10B6000003980068502100F033F820E003980068A8
:10B61000029A5168D26803F013FB03980068602116
:10B6200000F026F813E003980068029A5168D26887
:10B6300003F0DEFA03980068402100F019F806E0F4
:10B64000039800680299096800F012F8FFE703996F
:10B650003D220120885403993C220020885404A9EB
:10B660000020087004A8007805B000BD88FFCEFF58
:10B6700083B0029001910298806800900098074979
:10B680000840009001980099084307210843009062
:10B6900000980299886003B07047C0468FFFCFFFC3
:10B6A00085B00390029103983C21405C012803D1AE
:10B6B00004A90220087058E003993C220120885414
:10B6C00003993D2202208854039800684068019045
:10B6D00003980068806800900398006825498842B4
:10B6E00009D101980F21090588430190029841680A
:10B6F00001980843019001987021884301900298B5
:10B70000016801980843019001980399096848600D
:10B7100003980068174988420FD0039800680121F8
:10B720008907884209D0039800681349884204D0E9
:10B7300003980068114988420CD100988021884301
:10B74000009002988168009808430090009803993F
:10B750000968886003993D220120885403993C229E
:10B760000020885404A90020087004A8007805B0BF
:10B770007047C046002C01400004004000400140DA
:10B7800010B592B011900CA90020087011980068B3
:10B79000FD49884200D1FFE7119988680A69104382
:10B7A0004A691043C96908431090119800680068FD
:10B7B000F6490840109908431199096808601198E2
:10B7C000006840680321090388431199CA6810433F
:10B7D0000968486011988069109011980068EA49DA
:10B7E000884204D01198016A10980843109011986B
:10B7F00000688068E6490840109908431199096873
:10B80000886011980068C06A0F21884311994A6ABC
:10B8100010430968C86211980068DE49884227D140
:10B82000DD48006803210840099003281CD80998C6
:10B83000810001A04058874649B8000859B800085F
:10B8400051B8000861B800080EA9002008700EE089
:10B850000EA9022008700AE00EA90420087006E074
:10B860000EA90820087002E00EA91020087085E0DB
:10B8700011980068EC4988423AD1EE4800680C21E2
:10B88000084008900C282FD80898810001A0405843
:10B890008746C046C9B80008E9B80008E9B80008FA
:10B8A000E9B80008D9B80008E9B80008E9B8000804
:10B8B000E9B80008D1B80008E9B80008E9B80008FC
:10B8C000E9B80008E1B800080EA9002008700EE0F1
:10B8D0000EA9022008700AE00EA90420087006E0F4
:10B8E0000EA90820087002E00EA91020087045E09B
:10B8F00011980068CD49884203D10EA90020087034
:10B900003CE011980068CA49884203D10EA9002082
:10B91000087033E011980068C24988422BD1C548AD
:10B920000068032189020840079000280FD007987B
:10B9300001218902884212D007980121C902884258
:10B9400009D007980321890288420CD00FE00EA984
:10B95000002008700EE00EA9022008700AE00EA96F
:10B960000420087006E00EA90820087002E00EA965
:10B970001020087002E00EA91020087011980068CD
:10B98000A849884277D10EA800780690082826D8C2
:10B990000698810001A040588746C046C1B90008FA
:10B9A000DFB90008C9B90008DFB90008CFB900083D
:10B9B000DFB90008DFB90008DFB90008D7B900080F
:10B9C000FFF78EF90A900FE09B480A900CE0FFF712
:10B9D000FFF80A9008E00120C0030A9004E000206C
:10B9E0000A900CA9012008700A98002842D00A98F1
:10B9F0001199496A4A009149895A01F037FA0B9026
:10BA00000B9811994A6803215143884205D30B983A
:10BA1000119949680903884203D90CA901200870CB
:10BA200028E00A9811990491496A4A0083498A5A80
:10BA300000230593194601F03DFA049A059B040E74
:10BA4000090209190002526854080019594101F00D
:10BA500031FA0D900D98000A032808D30D98000DB7
:10BA6000002804D10D9811990968C86002E00CA95A
:10BA700001200870C5E01198C0690121C9038842FE
:10BA800061D10EA800780390082826D80398810079
:10BA900001A040588746C046BDBA0008DBBA00087E
:10BAA000C5BA0008DBBA0008CBBA0008DBBA000848
:10BAB000DBBA0008DBBA0008D3BA0008FFF710F9B8
:10BAC0000A900FE05C480A900CE0FFF781F80A90BA
:10BAD00008E00120C0030A9004E000200A900CA9AD
:10BAE000012008700A9800282CD00A981199029118
:10BAF000496A4A005149895A01F0B8F9029940004F
:10BB000049684A08801801F0B1F980B20D900D988B
:10BB1000102814D30DA84088002810D10D990F20AB
:10BB200081430FA801800D990E2211404A080F99F8
:10BB300011430180008811990968C86002E00CA9CE
:10BB4000012008705DE00EA800780190082830D828
:10BB50000198810001A040588746C04681BB00087B
:10BB6000B3BB00089DBB0008B3BB0008A3BB000823
:10BB7000B3BB0008B3BB0008B3BB0008ABBB0008F5
:10BB8000FFF7AEF80A9019E000800040F369FFCF9C
:10BB9000FFF4FF11003801405410024026480A907B
:10BBA0000CE0FFF715F80A9008E00120C0030A90A6
:10BBB00004E000200A900CA9012008700A980028CF
:10BBC0001FD00A9811990091496A4A001B49895A65
:10BBD00001F04CF9009949684A08801801F046F9CB
:10BBE00080B20D900D98102808D30DA84088002829
:10BBF00004D10D9811990968C86002E00CA90120D0
:10BC0000087011996A22012088521199682288527D
:10BC1000119900200867119948670CA8007812B0A4
:10BC200010BDC04600800040004400400048004075
:10BC3000004C0040541002400024F40064EE000860
:10BC400000B585B0039003998C2200208850FCF742
:10BC50001BFB0290039800680068000700280ED5BF
:10BC60000398029B1B49009101214905002202F023
:10BC700036F8002803D004A90320087025E00398B3
:10BC800000680068400700280ED50398029B114900
:10BC9000009101218905002202F021F8002803D03B
:10BCA00004A90320087010E0039984222020885002
:10BCB00003998822885003990020C866039980223E
:10BCC0000020885404A90020087004A8007805B05A
:08BCD00000BDC046FFFFFF01AB
:10BCD8008CB00490039102A80280049884214058F3
:10BCE800202800D09EE00398002803D002A80088EE
:10BCF800002803D105A90120087096E004988068FF
:10BD08000121090388420CD104980069002808D150
:10BD180003A80078C007002803D005A901200870EF
:10BD280083E004988021405C012803D105A9022002
:10BD380008707AE0049980220120885403980499B5
:10BD48000865029804995422885202980499562248
:10BD5800885204990020486704998C2288500499D5
:10BD68008422212088500498406E01214907884286
:10BD78002AD10498806801210903884207D10498D0
:10BD88000069002803D104992D48486702E0049906
:10BD98002A4848670499802200208854EFF31080CD
:10BDA80007900798019001220B920B9880F3108856
:10BDB800049801688868D2051043886001980A9041
:10BDC8000A9880F3108829E0049880680121090303
:10BDD800884207D104980069002803D104991648BD
:10BDE800486702E0049913484867049980220020B4
:10BDF8008854EFF31080069006980090012009906F
:10BE0800099880F310880498016808688022104314
:10BE1800086000980890089880F3108805A9002009
:10BE2800087002E005A90220087005A800780CB087
:10BE38007047C04649DE000815BF0008ADEC000891
:04BE48004DBE0008E3
:10BE4C008BB00490049884214058212857D1049831
:10BE5C006A21405A02A9088002A8008800284ED006
:10BE6C0004985621405A00282AD1EFF310800690EE
:10BE7C000698019001220A920A9880F3108804987F
:10BE8C0001688868D20590438860019809900998E8
:10BE9C0080F31088EFF31080059005980090012036
:10BEAC000890089880F3108804980168086840226C
:10BEBC001043086000980790079880F310881EE0E4
:10BECC0004980068C0690006002813D50498006D1A
:10BEDC000390039800880B4908400499096888620C
:10BEEC000499086D801C086504995622885A401ED6
:10BEFC008852FFE70298401E02A90880ACE70BB0FD
:08BF0C007047C046FF01000070
:10BF14008AB00390039884214058212842D1039881
:10BF24005621405A00282AD1EFF310800590059835
:10BF3400019001200990099880F310880398016802
:10BF4400086880229043086001980890089880F35C
:10BF54001088EFF31080049004980090012007905B
:10BF6400079880F3108803980168086840221043FA
:10BF7400086000980690069880F3108812E00398F1
:10BF8400006D0290029800880749084003990968E7
:10BF940088620399086D801C086503995622885AA3
:0CBFA400401E88520AB07047FF010000E8
:10BFB00000B589B00490039102A8028004988821FA
:10BFC0004058202856D10398002803D002A80088A2
:10BFD000002803D105A9012008704EE0049880686C
:10BFE0000121090388420CD104980069002808D176
:10BFF00003A80078C007002803D005A90120087015
:10C000003BE004988021405C012803D105A902206F
:10C01000087032E00499802201208854049900209D
:10C02000C86604980068174988421AD004980068C6
:10C0300040680002002814D5EFF31080069006989F
:10C04000019001220892089880F3108804980168F2
:10C05000086892061043086001980790079880F3DB
:10C0600010880498039902AA128800F00DF805A917
:10C07000087002E005A90220087005A8007809B040
:08C0800000BDC0460080004035
:10C0880093B00690059104A80280059806998865E2
:10C09800049806995C228852049806995E22885270
:10C0A80006990020086706988068012109038842DC
:10C0B8000DD106980069002804D1069960226448C9
:10C0C800885203E006996022FF20885229E00698EA
:10C0D800806800280DD106980069002804D10699C7
:10C0E8006022FF20885203E0069960227F20885250
:10C0F80017E0069880680121090788420DD1069843
:10C108000069002804D1069960227F20885203E044
:10C11800069960223F20885203E006996022002099
:10C12800885206998C22002088500699882222205D
:10C138008850EFF310800A900A9803900122129217
:10C14800129880F310880698016888681043886000
:10C1580003981190119880F310880698406E012179
:10C168004907884246D104A8008806996822895A56
:10C1780088423FDB0698806801210903884207D17D
:10C1880006980069002803D106993548086702E037
:10C198000699324808670699802200208854EFF3F0
:10C1A800108009900998029001221092109880F34B
:10C1B80010880698016808681202104308600298FF
:10C1C8000F900F9880F31088EFF31080089008986C
:10C1D800019001220E920E9880F31088069801684B
:10C1E800886812071043886001980D900D9880F3B5
:10C1F80010882AE00698806801210903884207D13F
:10C2080006980069002803D106991348086702E0D8
:10C218000699104808670699802200208854EFF391
:10C22800108007900798009001200C900C9880F3DC
:10C2380010880698016808680922520110430860AE
:10C2480000980B900B9880F31088002013B070476B
:10C25800FF010000FDDF0008D7DE0008FDC400086C
:04C268006DC200089B
:10C26C0000B59FB00F900F986021405A0DA908801F
:10C27C000F980068C06909900F98006800680890D2
:10C28C000F980068806807900F98882140582228E2
:10C29C0000D020E10F986821405A0BA908800BA808
:10C2AC00018800200029019005D009A800782021E0
:10C2BC000840400901900198C007002800D1CDE04A
:10C2CC000F980068406A0CA908800F98806D0E903A
:10C2DC000C980D9908400E9908800F99886D801C58
:10C2EC0088650F995E22885A401E88520F98006804
:10C2FC00C069099009A800784007002846D009A811
:10C30C000078C00700280DD008A84078C007002886
:10C31C0008D00F980068012303620F998C2288586B
:10C32C001843885009A80078800700280ED507A864
:10C33C000078C007002809D00F9801680220086215
:10C34C000F998C22885804231843885009A8007828
:10C35C00400700280ED507A80078C007002809D090
:10C36C000F980168042008620F998C2288580223C8
:10C37C00184388500F988C214058002806D00F98ED
:10C38C0002F0EAFC0F998C22002088500F985E2155
:10C39C00405A002861D1EFF3108014901498069045
:10C3AC0001221E921E9880F310880F98016808686D
:10C3BC0012029043086006981D901D9880F3108817
:10C3CC00EFF3108013901398059001201C901C988B
:10C3DC0080F310880F9801688868444A1040886080
:10C3EC0005981B901B9880F310880F9988222020A9
:10C3FC0088500F99002008670F98C06E012829D12A
:10C40C000F990020C866EFF31080129012980490D8
:10C41C0001201A901A9880F310880F980168086808
:10C42C0010229043086004981990199880F3108892
:10C43C000F980068C069102108400009012803D139
:10C44C000F980168102008620F985C21415A02F085
:10C45C0087FC02E00F9802F08DFC20E70F985E211C
:10C46C00415A0AA801800088002833D00AA8008805
:10C47C000F996822895A88422CDAEFF310801190B8
:10C48C001198039001221892189880F310880F9835
:10C49C000168886812079043886003981790179872
:10C4AC0080F310880F9910480867EFF310801090F4
:10C4BC001098029001201690169880F310880F980F
:10C4CC00016808682022104308600298159015989E
:10C4DC0080F3108805E00F980168886908221043E2
:10C4EC0088611FB000BDC046D7DE0008FEFFFFEF1D
:10C4FC0000B59DB00D900D986021405A0CA9088094
:10C50C000D980068C06908900D9800680068079045
:10C51C000D980068806806900D9888214058222854
:10C52C0000D01EE10D986821405A0AA908800AA87B
:10C53C00018800200029009005D008A8007820214F
:10C54C000840400900900098C007002800D1CBE0BB
:10C55C000D980068406A0BA908800B980C9908404C
:10C56C000D99896D08700D99886D401C88650D9921
:10C57C005E22885A401E88520D980068C069089047
:10C58C0008A800784007002846D008A80078C00703
:10C59C0000280DD007A84078C007002808D00D98B7
:10C5AC000068012303620D998C2288581843885027
:10C5BC0008A80078800700280ED506A80078C007C8
:10C5CC00002809D00D980168022008620D998C2270
:10C5DC00885804231843885008A80078400700287E
:10C5EC000ED506A80078C007002809D00D98016860
:10C5FC00042008620D998C22885802231843885015
:10C60C000D988C214058002806D00D9802F0A4FB00
:10C61C000D998C22002088500D985E21405A0028DC
:10C62C0061D1EFF3108012901298059001221C92A8
:10C63C001C9880F310880D980168086812029043CA
:10C64C00086005981B901B9880F31088EFF31080FE
:10C65C0011901198049001201A901A9880F3108868
:10C66C000D9801688868444A1040886004981990B5
:10C67C00199880F310880D998822202088500D99E4
:10C68C00002008670D98C06E012829D10D99002053
:10C69C00C866EFF31080109010980390012018904A
:10C6AC00189880F310880D98016808681022904340
:10C6BC00086003981790179880F310880D980068FD
:10C6CC00C069102108400009012803D10D980168A8
:10C6DC00102008620D985C21415A02F041FB02E0E7
:10C6EC000D9802F047FB22E70D985E21415A09A8EC
:10C6FC0001800088002833D009A800880D99682291
:10C70C00895A88422CDAEFF310800F900F98029020
:10C71C0001221692169880F310880D98016888688B
:10C72C0012079043886002981590159880F3108832
:10C73C000D9910480867EFF310800E900E98019039
:10C74C0001201490149880F310880D9801680868E3
:10C75C0020221043086001981390139880F31088DE
:10C76C0005E00D98016888690822104388611DB0A6
:0CC77C0000BDC046FDDF0008FEFFFFEF1F
:10C7880000B587B00590049103920293059800289C
:10C7980003D106A90120087052E005988421405869
:10C7A800002806D105998022002088540598FAF7B8
:10C7B8005FFB059984222420885005980168086841
:10C7C8000122904308600598FEF7D6FF012803D19F
:10C7D80006A90120087033E00598806A002802D075
:10C7E800059801F0DDF9059801688868012293032E
:10C7F80018438860059800688068D10388430499C5
:10C8080008430599096888600398400501900298D3
:10C8180001040198084301900598006800680A49D6
:10C828000840019908430599096808600598016856
:10C838000868104308600598FFF7FEF906A9087014
:0CC8480006A8007807B000BDFFFF00FC50
:10C8540070B58AB009900998406E002807D10999EB
:10C864006A220120885209996822885232E008A974
:10C8740001910820087007A9087009980068806869
:10C88400072252061040400E06AA02921070099820
:10C8940000688068420F05A80270097802780E4883
:10C8A4000490805C48430D490391895C00F0DCFAF4
:10C8B400019B029A039904460498099D6A26AC5385
:10C8C4001B781278805C5843895C00F0CDFA099992
:10C8D400682288520AB070BD4DF8000855F8000867
:10C8E40070B5FFB0FFB098B0FFAB283305930B468B
:10C8F40005990693034606980B63C8628A6209A8E1
:10C904000861012080024861002088610A6B0A6284
:10C91400C861059AD06A0178FFA84C300170D16AC9
:10C92400491CD1620078002800D17EE1FFA84C3078
:10C934000078252800D06CE105990020486001208A
:10C94400C8600598C06A0178FFA84C30017000786F
:10C95400233804900D2845D80498810001A040583C
:10C964008746C046D7C90008E9C90008E9C90008D4
:10C97400E9C90008E9C90008E9C90008E9C90008CB
:10C98400E9C90008C5C90008E9C90008A1C9000827
:10C99400E9C90008E9C90008B3C90008059948684D
:10C9A400012210434860C86A401CC8621DE0059912
:10C9B4004868022210434860C86A401CC86214E0F8
:10C9C40005994868042210434860C86A401CC8623C
:10C9D4000BE005994868082210434860C86A401C67
:10C9E400C86202E005990020C8600598C068002864
:10C9F400A7D10599002008600598C06A0178FFA8AE
:10CA04004C3001700078302804DBFFA84C300078EB
:10CA14003A2800DB0FE00599C86A401CC862086820
:10CA24000A224243FFA84C3000788018303808604E
:10CA340001200028E0D1059800218160C06A0178B6
:10CA4400FFA84C30017000782E2822D10599C86ABD
:10CA5400401CC8620598C06A0178FFA84C30017078
:10CA64000078302804DBFFA84C3000783A2800DB3B
:10CA74000FE00599C86A401CC86288680A224243CC
:10CA8400FFA84C30007880183038886001200028D6
:10CA9400E0D10598C06A0078FFA94C310870FFA85E
:10CAA4004C3000786C2804D0FFA84C3000786828FB
:10CAB40009D10598C16A491CC162C06A0078FFA9FE
:10CAC4004C31087000E002E001200028E7D1FFA803
:10CAD4004C3000780390252800D18FE00398582823
:10CAE40048D0039863280FD0039864281CD0039877
:10CAF400702871D0039873284FD00398752826D0D6
:10CB04000398782836D07FE00598836A19680A1D4F
:10CB14001A600968C160C16808A801700178FFA89B
:10CB2400383002F065F96FE0059A936A1868011DC0
:10CB340019600068D060D1689368106852680192E7
:10CB44000090FFA838300A2201F069FB5CE0059AE6
:10CB5400936A1868011D19600068D060D1689368F1
:10CB64001068526801920090FFA838300A2200F041
:10CB740075F849E0059A936A1868011D1960006800
:10CB8400D060D16893681068526801920090FFA841
:10CB94003830102200F062F836E00598826A106896
:10CBA400011D11600068079007980178FFA84C30B8
:10CBB40001700799491C07910078002800D10AE008
:10CBC400FFA84C300178FFA8383002F011F905981D
:10CBD400C0690028E8D517E00598836A19680A1D1A
:10CBE4001A600968C160C16800200190082300939D
:10CBF400FFA83830102200F031F805E0FFA83830E3
:10CC0400252102F0F5F8FFE70599C86A401CC862BF
:10CC140006E0FFA84C300178FFA8383002F0E8F8AD
:10CC24000598C069002800D473E60598C0690128F6
:10CC34000EDB05988069002805D00599086B8A6980
:10CC440009A900F06BFA05998A69C8698018C86156
:0CCC54000598C0697FB07FB018B070BDBB
:10CC600010B590B0139C129C0F900E910D920C93E6
:10CC70000E98099001200A90089009980D99884211
:10CC800008D309980D9900F0F1F809900898401C14
:10CC90000890F2E70C980899884201D90C980890FE
:10CCA00013A80078C007002834D11298002831D08A
:10CCB00013A800788007002806D50C98002803D117
:10CCC00007A93020087002E007A9202008701299F7
:10CCD0000020002906900BD00899129A0120002309
:10CCE00004939142059001D304980590059806900D
:10CCF0000698C00700280DD01298401E12900F9879
:10CD000007A9097802F076F80F98C068002800D5C6
:10CD100000E0DCE70F98C06800285DD40C9802287A
:10CD200003D30C98401E0C9009E00E980A9900F06D
:10CD30009DF80B900B980D99884200D204E00D9855
:10CD40000A9948430A90E9E70E980A9900F08EF88C
:10CD50000B900B980A9941430E98401A0E900F9829
:10CD60000B9A1E49895C02F045F80F98C0680028AC
:10CD700000D507E00D990A9800F078F80A900A9813
:10CD80000028E1D113A80078C007002824D0129809
:10CD9000002821D012990020002903900BD0089977
:10CDA000129A0120002301939142029001D301982D
:10CDB0000290029803900398C00700280CD01298A4
:10CDC000401E12900F98202102F014F80F98C068AE
:10CDD000002800D500E0DDE710B010BD5DF80008C8
:10CDE0004A0010D2520D03231B02FF33D21A0AD479
:10CDF00052421F3209D4400DC90208430123DB0708
:10CE00001843D040704700207047D0177047C04685
:10CE100042221201033A010007D002D4013A00185D
:0CCE2000FCD51205C30A400599187047A4
:10CE2C00CA1751408B1A17D0C1174A409446484034
:10CE3C00411A48081A0000E052008242FCD9002036
:10CE4C0000E05208914200D3891A40419A42F8D12D
:10CE5C0062465040801A704710B500F075F810BD4E
:10CE6C000A0015D00300400800E052008242FCD9B1
:10CE7C00002000E052089B1A06D340418A42F9D1A7
:10CE8C00704752089B18F8D200188A42F9D17047A3
:08CE9C0010B500F059F810BDBB
:10CEA40038B504004D42FFF7DFFF4543611938BD33
:10CEB400002B09D1002907D110B51100FFF7F0FFAD
:10CEC4000A000021002310BD70B400240125ED07E1
:10CED400002B07D1002905D0834203D2130000227E
:10CEE4002C0000250026A419994200D1904212D9A1
:10CEF40092185B4103D2EE076D086408F3E7DE077E
:10CF04005B08520892190126F6079B1903E0DE0715
:10CF14005B0852089219801A994103D364416D4108
:10CF2400F5D30FE024196D410AD2DE075B085208DD
:10CF3400921980185941F5D364416D41E7D301E05A
:10CF44008018594102000B002000290070BC704772
:08CF5400002000217047C046D7
:10CF5C00411C02780130002AFBD1401A7047C046B0
:10CF6C00002A03D0013A8B5C8354FBD17047C04636
:10CF7C0000220B0011001A00002A02D0013A815441
:04CF8C00FCD170471D
:10CF900003231048104A03614361104B8261C3614F
:10CFA0008023DB000362002383624362C362026664
:10CFB0000B4A53214266102282660367094AC36600
:10CFC000436700E0D17BC1540133013A102BF9D102
:10CFD0007047C0464C0D002064D3000810070020A5
:08CFE000F005002080D30008D9
:10CFE800F8B54746CE46C568836804004068994648
:10CFF8005B1B80B50E00170098464019934207D96D
:10D00800FFF7B0FFED19E560C0BCB946B046F8BD02
:10D018001A00FFF7A7FF4B463100ED19ED1A2A0059
:0CD0280060684144FFF79EFFEDE7C04642
:10D03400F8B54746CE46002380B58846070016005B
:10D044009946C56884681BE0013B5B1B641BB442C2
:10D0540000D934009C4200D91C0078682200414663
:10D064004019FFF781FF2D19A144A044361BBC6869
:10D07400631B5A1E93415B421D40FD60002E06D087
:10D084003B699D42E0D3013B1B195B1BDEE748462D
:08D09400C0BCB946B046F8BD6E
:10D09C0070B50600431C5C00E418E00074001C4BE7
:10D0AC00A419E400C0181B19DC6A1500012C06D069
:10D0BC00022C1FD0002C10D00024200070BD9A6AC6
:10D0CC005C6AA2421FD9013A121B2C00954200D96E
:10D0DC0014002200FFF782FFEFE79A6A5E6AB24201
:10D0EC000CD9013A961BB542E7D82A00FFF776FF18
:10D0FC002C00E2E7FFF798FF0400DEE71B6AD2186A
:10D10C00013A961BEFE71B6AD218013A121BDCE7B7
:04D11C004C0D002096
:10D12000F8B50B4B04001B780D001600002B0CD03B
:10D13000EFF31087012181F31088320029002000CD
:10D14000FFF7ACFF87F31088F8BDFFF721FFEFE78B
:04D150004C0D002062
:10D15400F8B5050008000C00FFF7FEFE0A4B0600B8
:10D164001B78002B0CD0EFF31087012181F310887A
:10D17400320021002800FFF78FFF87F31088F8BDE5
:0CD18400FFF704FFEFE7C0464C0D002051
:08D190000A000000B80B0000CA
:08D1980001000000640000002A
:08D1A0000A000000B80B0000BA
:08D1A80001000000640000001A
:08D1B0000A000000B80B0000AA
:08D1B80001000000640000000A
:08D1C0000A000000B80B00009A
:08D1C8000100000064000000FA
:10D1D0000A000000B80B0000B80B0000B80B0000FC
:10D1E0000100000064000000640000006400000012
:10D1F0000A000000B80B0000B80B0000B80B0000DC
:10D2000001000000640000006400000064000000F1
:10D21000004B0000650001000100E8030000000071
:10D2200000009600CC00DC0568024803A40620023A
:04D2300000000000FA
:10D23400034C206804348047FBE7F6F7E3FAFEE783
:04D2440070F8000876
:04D24800D1300008D9
:10D24C0087B006900591049203A9002008701F2056
:10D25C0002900299481E029000200029019009D0EA
:10D26C00059802991F221140C840012108404142F3
:10D27C00484101900198C007002800D0E9E70498C4
:10D28C00009018284CD80098810001A0405887467F
:10D29C002BD300082DD300082DD300082DD3000864
:10D2AC002DD300082DD300082DD300082DD3000852
:10D2BC001DD300082DD300082DD300082DD3000852
:10D2CC002DD300082DD300082DD300082DD3000832
:10D2DC000FD300082DD300082DD300082DD3000840
:10D2EC002DD300082DD300082DD300082DD3000812
:10D2FC0001D300080298072802D303A90120087063
:10D30C0011E00298082802D303A9012008700AE052
:10D31C000298102802D303A90120087003E002E050
:10D32C0003A90120087003A8007800280DD10598E6
:10D33C000699096848610698006880681821884336
:10D34C000499084306990968886003A8007807B017
:02D35C00704718
:06D35E00F5F7AFFE67E7E2
:09D364005465726D696E616C0084
:10D36D004465766963652049443A20756E6B6E6F2E
:03D37D00776E00C8
:10D3800000000000000054545220524547474553C6
:01D39000009C
:10D39100547279696E6720746F207265737461725B
:03D3A100742E00E7
:02D3A400FEE7A2
:02D3A600FEE7A0
:02D3A800FEE79E
:02D3AA00FEE79C
:02D3AC00FEE79A
:02D3AE00FEE798
:02D3B000FEE796
:02D3B200FEE794
:02D3B400FEE792
:02D3B600FEE790
:02D3B800FEE78E
:02D3BA00FEE78C
:02D3BC00FEE78A
:02D3BE00FEE788
:02D3C000FEE786
:02D3C200FEE784
:02D3C400FEE782
:02D3C600FEE780
:02D3C800FEE77E
:02D3CA00FEE77C
:02D3CC00FEE77A
:02D3CE00FEE778
:02D3D000FEE776
:02D3D200FEE774
:10D3D40010B596B008A803903821FFF7CDFD0020C2
:10D3E400019007900690059004900120029040025D
:10D3F400FCF7B2FF019A029903980B2308930B04DC
:10D4040009930B020B930323DC020C9440240D9428
:10D414000E9102240F9410931192102212924A0436
:10D4240013924A06149249071591FCF7CFFF00287E
:10D4340001D0F8F7EDFA07200490022105910020AD
:10D444000690079004A8FDF7B5FA002801D0F8F774
:0AD45400DFFAFDF75FFC16B010BD13
:10D45E0000B587B006AB1880059104A802800020A5
:10D46E000390039806A90988884218DA059804A93A
:10D47E0001910988012201F07EFBFF204E300290BF
:10D48E00FAF701FF019905980988002201F073FB54
:10D49E000298FAF7F8FE0398401C0390E1E707B0F4
:02D4AE0000BDBF
:10D4B00030B587B004460D980C9D0B9D0A9D0694CF
:10D4C00005910492039302A90880FAF7DDFE01900A
:10D4D000059800680399884248D204980068009033
:10D4E000002806D00098012811D00098022827D0E3
:10D4F0003BE00C9802A90988012201F043FB019846
:10D500000699086004990868401C08602DE001989D
:10D5100006990968401A0A99059A12685200895AB0
:10D5200088420CD90C9802A90988002201F02AFB34
:10D5300001980699086004990868401C086014E086
:10D54000019806990968401A0B99059A12685200C9
:10D55000895A884209D901980699086004990020DF
:10D56000086005990868401C086002E005990020E1
:06D57000086007B030BDA9
:02D576007047FC
:02D578007047FA
:10D57A0000B581B000900098016808684022904385
:10D58A00086000998422202088500099002048676A
:0AD59A00009801F0ECFB01B000BDA9
:10D5A40000B581B00090009926220C208854009A7E
:10D5B4001068FF21283151188B239B00D25AFEF7A3
:06D5C40089FB01B000BD6F
:10D5CA0081B0009000998B2082000020885001B021
:02D5DA00704798
:10D5DC0081B0009000994520C2000020885000992D
:06D5EC00087501B0704754
:10D5F20010B588B00A9C07900691059204A80370A2
:10D6020006984078039003980190032806D0019869
:10D6120006280CD00198102814D01EE0079806990D
:10D62200059A04AB1B78F9F7BCFF02901CE007983F
:10D632000699059A04AB1B780A9C0094FAF727F81E
:10D64200029011E007980699059A04AB1B780A9C90
:10D652000094FAF7A4F8029006E007980399059B54
:0ED66200012200F004F80290029808B010BDFA
:10D6700084B003900291019200930298803002904E
:10D6800002980399009A88540098401C00900198D1
:10D690000399009A88540098401C0090009804B0A8
:02D6A0007047D1
:06D6A200F920C0007047F2
:10D6A80081B000900098806804210840800801B08B
:02D6B8007047B9
:10D6BA0083B002900191009202984069019A042174
:10D6CA000A400721914088430099914008430299F2
:06D6DA00486103B0704737
:10D6E00000B583B0019001980068FFF7DDFF0028C6
:10D6F0002CD00198006800F0C9F8002803D10198E7
:10D700000068FBF7FFFDFAF7BFFD00900198006885
:10D7100080684007002819D5FAF7B6FD0099401A2D
:10D72000032812D3019800688068400700280CD5B0
:10D730000199886D102210438865019AD16D0120EE
:10D740000143D16502A9087003E0DFE702A90020C8
:0AD75000087002A8007803B000BDC5
:10D75A0000B583B0019001985421405C012803D19F
:10D76A0002A90220087024E0019954220120885459
:10D77A000198FFF7B0FF014668460170007800285B
:10D78A0010D1019801F001F801466846017000784D
:10D79A00002807D10198806D0121084309028843B6
:10D7AA00019988650199542200208854009802A999
:0AD7BA00087002A8007803B000BD5B
:10D7C40081B000900098C06803218902084041425A
:06D7D400484101B070475E
:10D7DA0000B583B002900298806A0190019801F026
:06D7EA00E6F803B000BDEB
:10D7F00000B583B002900298806A01900199886D0B
:10D800004022104388650199C86D04221043C86501
:0AD81000019801F0CDF803B000BD4F
:10D81A0083B00290019100920298806A019A1F21B6
:10D82A000A400F2319469140884300999B061940E4
:0ED83A00890E914008430299886203B070473E
:10D8480081B000900098006807218905084001B060
:02D85800704717
:0ED85A0081B0009000998020086001B07047F6
:10D8680081B000900099486880221043486001B058
:02D878007047F7
:10D87A0081B000900099486880229043486001B0C6
:02D88A007047E5
:10D88C0081B000900098806802210840400801B0E7
:02D89C007047D3
:10D89E0000B581B001466846017000214056FBF785
:06D8AE00FCFD01B000BD0D
:10D8B40000B581B001466846017000214056FBF76F
:06D8C40005FE01B000BDED
:10D8CA0000B583B001900198002803D102A9012074
:10D8DA00087014E001980079002805D10199002008
:10D8EA0048710198F5F73BFE0199022008710199E8
:10D8FA0000200861019A0121117102A9087002A889
:06D90A00007803B000BD2F
:10D9100082B00190009101980068806B00991022FC
:0ED9200011401F228A401040C84002B07047DC
:10D92E0000B587B0059004910392029301A90020DF
:10D93E00087005982421405C012803D106A9022015
:10D94E00087030E00599242201208854059825217D
:10D95E00405C01281AD10599252202208854059988
:10D96E000020C86305980168086801220092904360
:10D97E00086005980499039A029BFCF70AF8009A2E
:10D98E000598016808681043086009E00599802031
:10D99E00C863059924220020885401A9012008702B
:0ED9AE00019806A9087006A8007807B000BD11
:10D9BC0000B587B0059004910392029301A9002051
:10D9CC00087005982421405C012803D106A9022087
:10D9DC0008705EE0059924220120885405982521C1
:10D9EC00405C012848D105992522022088540599CC
:10D9FC000020C863059801680868012290430860FC
:10DA0C0005980499039A029BFBF7C4FF0598006BD9
:10DA1C00002806D00598016808680E22104308609B
:10DA2C000BE005980168086804229043086005988B
:10DA3C00016808680A22104308600598406C006869
:10DA4C00C003002806D50598416C08680122120213
:10DA5C00104308600598006D002806D00598016DEC
:10DA6C0008680122120210430860059801680868D2
:10DA7C0001221043086009E005998020C8630599CC
:10DA8C0024220020885401A901200870019806A9BD
:0ADA9C00087006A8007807B000BD6E
:10DAA60084B0009101460098039102A9088003986A
:10DAB60000690988084203D001A90120087002E024
:0EDAC60001A90020087001A8007804B0704784
:02DAD400704799
:02DAD600704797
:10DAD80000B583B001900198002803D102A9012064
:10DAE80008703EE001983D21405C002806D101996C
:10DAF8003C22002088540198F9F7DEF801993D226C
:10DB080002208854019901C9FDF796FA0199482223
:10DB18000120885401993E220120885401993F220E
:10DB280088540199402288540199412288540199C6
:10DB380042228854019943228854019944220120A1
:10DB4800885401994522885401994622885401999C
:10DB58004722885401993D220120885402A90020B7
:0ADB6800087002A8007803B000BDA9
:10DB720085B004900391029201930498806800900A
:10DB82000098FF2109028843009003990298019AA4
:10DB92001202104301430098084300900098049930
:06DBA200886005B0704729
:10DBA80081B0009000982821405CC00700280AD066
:10DBB8000098006840680121490488430099CA6AAE
:10DBC80010430968486000982821405C80070028B5
:10DBD8000AD5009800684068012109048843009923
:10DBE8000A6B10430968486000982821405C400788
:10DBF80000280AD5009800684068012189048843F4
:10DC080000994A6B10430968486000982821405CD5
:10DC1800000700280AD50098006840680121C90358
:10DC2800884300998A6B1043096848600098282146
:10DC3800405CC00600280AD5009800688068012169
:10DC4800090388430099CA6B1043096888600098E3
:10DC58002821405C800600280AD500980068806862
:10DC680001214903884300990A6C104309688860B8
:10DC780000982821405C4006002819D500980068C3
:10DC88004068012109058843009A536C18431268BB
:10DC980050600098406C88420AD10098006840683B
:10DCA80003214905884300998A6C10430968486034
:10DCB80000982821405C000600280AD500980068D2
:10DCC80040680121C90488430099CA6C1043096857
:06DCD800486001B0704736
:10DCDE0010B596B0189C0890079106A8027005938F
:10DCEE0008980068C06907990840401A41424841A7
:10DCFE0006A90978884200D098E01898401C0028A0
:10DD0E0000D192E0FAF7B9FA0599401A18998842AB
:10DD1E0002D81898002838D1EFF310800D900D9886
:10DD2E00049001201590159880F3108808980168CA
:10DD3E0008680D22520190430860049814901498BC
:10DD4E0080F31088EFF310800C900C980390012252
:10DD5E001392139880F3108808980168886890438E
:10DD6E00886003981290129880F310880899842284
:10DD7E0020208850089988228850089980220020F7
:10DD8E00885409A90320087053E0089800680068B9
:10DD9E004007002849D508980068C0690121C902CA
:10DDAE000840C00A012840D1089801680120C0022D
:10DDBE000862EFF310800B900B98029001201190E7
:10DDCE00119880F310880898016808680D22520196
:10DDDE009043086002981090109880F31088EFF32B
:10DDEE0010800A900A98019001220F920F9880F3EA
:10DDFE0010880898016888689043886001980E9092
:10DE0E000E9880F310880899842220208850089953
:10DE1E008822885008998C228850089980220020E8
:10DE2E00885409A90320087003E059E709A90020C6
:0ADE3E00087009A8007816B010BDA6
:10DE480089B0029002988421405821283DD1029837
:10DE58005621405A00282AD1EFF3108004900498E4
:10DE6800019001200890089880F3108802980168B2
:10DE7800086880229043086001980790079880F30B
:10DE88001088EFF31080039003980090012006900B
:10DE9800069880F3108802980168086840221043A9
:10DEA800086000980590059880F310880DE00299A5
:10DEB800086D0078096888620299086D401C086539
:0EDEC80002995622885A401E885209B07047AF
:10DED60000B591B0079007986021405A05A90880BF
:10DEE600079888214058222800D07CE007980068CF
:10DEF600406A04A908800798806D069004980599E1
:10DF06000840069908800799886D801C8865079ADD
:10DF16005E21505A401E50520798405A002861D13F
:10DF2600EFF310800A900A98039001201090109841
:10DF360080F3108807980168086809225201904307
:10DF4600086003980F900F9880F31088EFF3108005
:10DF560009900998029001220E920E9880F310887B
:10DF66000798016888689043886002980D900D981C
:10DF760080F310880799882220208850079900206E
:10DF860008670798C06E012829D107990020C8663E
:10DF9600EFF3108008900898019001200C900C98DF
:10DFA60080F310880798016808681022904308607B
:10DFB60001980B900B9880F3108807980068C06949
:10DFC600102108400009012803D107980168102094
:10DFD600086207985C21415A00F0C5FE02E00798E6
:10DFE60000F0CBFE05E00798016888690822104317
:06DFF600886111B000BDBE
:10DFFC0000B58FB0059005986021405A04A908809F
:10E00C00059888214058222800D07AE005980068AD
:10E01C00406A03A908800398049908400599896D02
:10E02C0008700599886D401C8865059A5E21505AC8
:10E03C00401E50520598405A002861D1EFF31080D1
:10E04C0008900898029001200E900E9880F310888A
:10E05C0005980168086809225201904308600298EB
:10E06C000D900D9880F31088EFF3108007900798AF
:10E07C00019001220C920C9880F31088059801688D
:10E08C0088689043886001980B900B9880F31088F7
:10E09C00059988222020885005990020086705984A
:10E0AC00C06E012829D105990020C866EFF31080B5
:10E0BC0006900698009001200A900A9880F3108828
:10E0CC000598016808681022904308600098099030
:10E0DC00099880F3108805980068C06910210840E1
:10E0EC000009012803D105980168102008620598E1
:10E0FC005C21415A00F034FE02E0059800F03AFE33
:10E10C0005E00598016888690822104388610FB002
:02E11C0000BD44
:10E11E0000B585B00390029103988021405C0128E0
:10E12E0003D104A9022008702FE003998022012058
:10E13E008854039984220092242088500398006802
:10E14E0000680190039801680868012290430860F6
:10E15E00039800688068072149078843029908439D
:10E16E000399096888600398FEF76DFB009A019881
:10E17E00039909680860039920208850039980222A
:10E18E000020885404A90020087004A8007805B067
:02E19E0000BDC2
:10E1A00000B585B00390029103988021405C01285E
:10E1B00003D104A9022008702FE0039980220120D6
:10E1C0008854039984220092242088500398006880
:10E1D0000068019003980168086801229043086074
:10E1E000039800688068072149068843029908431C
:10E1F0000399096888600398FEF72CFB009A019840
:10E2000003990968086003992020885003998022A7
:10E210000020885404A90020087004A8007805B0E4
:02E2200000BD3F
:10E2220030B58FB0139C129C0E900D910C920B93F3
:10E232000D98002803D50D984042089001E00D98F2
:10E2420008900898099001200A9009980C99884230
:10E2520008DB09980C99FEF7E8FD09900A98401C22
:10E262000A90F2E70B980A99884201D90B980A9012
:10E27200129800280AD00D98002804D413A8007818
:10E282004007002802D51298401E129013A8007869
:10E292008007002802D50B98002829D013A80078FF
:10E2A200C007002824D11298002821D012990020FA
:10E2B200002907900BD00A99129A01200023059396
:10E2C2009142069001D30598069006980790079808
:10E2D200C00700280CD01298401E12900E982021E0
:10E2E20000F087FD0E98C068002800D500E0DDE749
:10E2F2000E98C068002858D40D98002807D50D98AC
:10E3020040420D900E982D2100F073FD09E013A8F4
:10E3120000784007002804D50E982B2100F069FDF3
:10E32200FFE70E98C06800283FD413A80078800742
:10E3320000282CD513A80078C007002827D10B98F5
:10E34200002824D11298002821D0129900200029F7
:10E3520004900BD00A99129A012000230293914251
:10E36200039001D302980390039804900498C00785
:10E3720000280CD01298401E12900E98302100F006
:10E3820038FD0E98C068002800D500E0DDE70E9841
:10E39200C068002809D40E980D990C9A0B9B129C08
:0EE3A200139D01950094FEF75AFC0FB030BD9C
:10E3B00082B000B585B0079306920490039106A839
:10E3C00001900498039901AAFEF78CFA0290029832
:0AE3D00005B002BC02B08E46704793
:10E3DA0008D1002806D1F54204D801D3002A01D178
:10E3EA006D0D09D10020C143090DC904F0BDF9D151
:10E3FA001242F7D1640DF5D00020C14349054908FE
:10E40A00A6E000206146F0BDF0B50127FF070E0027
:10E41A005E403E40B446BE0A4C18DD18F442D7D2DC
:10E42A00F542E4D2640DECD06D0DEAD06419C9024C
:10E43A003943460DC0023143DB023B43DB0A10B4C9
:10E44A008E4685B297B26F43140C6C433E0CA419E6
:10E45A00260C2404BFB227439CB26C43A419190C9E
:10E46A006943250CA4B249190D04090C6419000C5E
:10E47A0095B245433E0C76193743BFB2360C150C9C
:10E48A004543AD19A6B2240CAD192E0437432E0C00
:10E49A0036199DB24543AD19ACB22E0C89191D0C23
:10E4AA0045436D182E04290C3443704680B295B248
:10E4BA0045433E0C76193743BFB2360C150C45431B
:10E4CA00AD19A6B2AD19240C2E0437432E0C3619F9
:10E4DA009DB24543AD19ACB22E0C89191D0C4543AA
:10E4EA006D182E043443290C75462D0C90B26843DE
:10E4FA003E0C80190604BFB23E43070CA0B23F1877
:10E50A00120C6A43D019020C80B2240CA4189AB2D5
:10E51A006A43121914042043120C89181B0C6B430A
:10E52A00C91810BC01273D05294203D1B61940413B
:10E53A004941013CFF077D0D013D641B0BDB6D006A
:10E54A00AC4209DA240500254208BE41684161410E
:0AE55A0066463143F0BD54E74EE77A
:10E5640030B589B00D9C0C9C0890079106920593D8
:10E574000698002802D00698012802D101200390B1
:10E5840001E00220039003980930049006980028C3
:10E5940002D00698012802D10498401C04900898DF
:10E5A4000599079A069B039C049D01950094F8F72E
:10E5B40027FD0899002048770899888408990884D9
:10E5C400089926228854089908770899C8830899D5
:10E5D400222288540C9808998D22920088500D9814
:0CE5E40008994722D200885009B030BDD1
:10E5F00081B00090009884214058212820D10098B3
:10E600005621405A00280CD10098016808688022E1
:10E610009043086000980168086840221043086031
:10E620000DE00099086D0078096888620099086D0E
:10E63000401C086500995622885A401E88520BE0FB
:10E64000009801680868802290430860009801687B
:0CE65000086840221043086001B07047C9
:10E65C0000B585B00490039104980399891EF8F7CE
:10E66C0025FF014601A80180049A03998A18511EBE
:10E67C0009780902921E12788A1869460A80008865
:10E68C000988884202D10398029002E00020C0431E
:08E69C000290029805B000BDD8
:10E6A40000B585B00490039104980399F8F702FF2C
:10E6B400014602A80180029901AA117040786946B6
:10E6C400087001980499039A88540398401C039095
:10E6D40000980499039A88540398401C0390039863
:04E6E40005B000BDC0
:10E6E80081B000900098007D0121084001B070477A
:10E6F80010B586B005900020049005982730039047
:10E708000598FEF75EFF03980178059AFF202830E8
:10E71800029011540499491C0491059C20180399EE
:10E72800049A0B780094FEF760FF0299049005980C
:10E7380040180499FFF7B2FF0490049805998B22BA
:10E74800920088500598FEF729FF0598FEF742FFCA
:04E7580006B010BD3A
:10E75C0000B581B000900098F9F70EFDF9F7FCFCBC
:04E76C0001B000BD3B
:10E7700081B0009000988068012109070840000FCF
:04E7800001B070472D
:10E7840081B00090009880680121084001B0704772
:10E7940000B585B0039003980068FFF775F8019001
:10E7A40003980068FFF7ECFF002842D00198002886
:10E7B4003FD103980068806805210840012808D1EA
:10E7C40003980068FAF770F803980168032008605A
:10E7D4000CE00399886D102210438865039AD16D6B
:10E7E40001200143D16504A9087025E0F9F74AFD29
:10E7F4000290039800688068C007002819D0F9F7D0
:10E8040041FD0299401A032812D3039800688068D6
:10E81400C00700280CD00399886D10221043886526
:10E82400039AD16D01200143D16504A9087003E066
:10E83400DFE704A90020087004A8007805B000BD33
:10E8440000B583B002900298806A01900198806DAF
:10E854005021084238D10199886D01225202104397
:10E86400886501980068FEF7ABFF002828D001985E
:10E87400807E002824D101980068006800070028E1
:10E884001ED501980068FEF70DFF00280ED10198EF
:10E89400016848680C22904348600198806D01210A
:10E8A4000843090288430199886509E00199886D44
:10E8B4002022104388650199C86D01221043C86560
:10E8C400019800F06FF80DE00198806DC0060028F3
:10E8D40003D5019800F06AF804E00198006D416BDB
:08E8E4000298884703B000BD53
:10E8EC0000B583B0019001985421405C012803D1FC
:10E8FC0002A9022008704DE001995422012088548D
:10E90C000198FEF7E7FE0146684601700078002882
:10E91C0039D10198006D2521405C02280ED1019857
:10E92C00006DFBF76FF8014668460170007800280F
:10E93C0004D00199886D40221043886501980168C4
:10E94C00486810229043486068460078002805D13A
:10E95C000198FFF719FF6946087002E00198FFF76C
:10E96C0013FF68460078002807D10198806D0121BB
:10E97C000843090288430199886501980168C868B1
:10E98C0001229043C86001995422002088540098B9
:0CE99C0002A9087002A8007803B000BDBA
:08E9A80081B0009001B070473E
:08E9B00081B0009001B0704736
:08E9B80081B0009001B070472E
:10E9C00082B0019000910198006807218905884371
:0CE9D000009908430199086002B07047EC
:10E9DC0081B00090009901200002086001B07047DE
:10E9EC0081B00090009948680122120210434860DF
:04E9FC0001B07047AF
:10EA000081B000900099486801221202904348604A
:04EA100001B070479A
:10EA140081B00090009901204002086001B0704765
:10EA240081B0009000994868012252021043486066
:04EA340001B0704776
:10EA380081B00090009948680122520290434860D2
:04EA480001B0704762
:10EA4C0081B00090009880680121084001B07047A7
:10EA5C0081B0009000988068C00F401E4142484130
:04EA6C0001B070473E
:10EA700081B0009000980068B42140587F21084080
:04EA800001B070472A
:10EA840000B583B0034602A80370019100920021EF
:0CEA940040560199FAF7C6FC03B000BD23
:04EAA000FAF72EFD56
:10EAA40000B581B000900098FAF736FD01B000BDC2
:10EAB40083B00190009101984079012803D102A903
:10EAC400022008703AE0019901204871019902205E
:10EAD40008710098102108400122824001980168C1
:10EAE400086810430860009800280DD10198006858
:10EAF40000683E210840022805D101980168486851
:10EB040001221043486010E00198006800681F214A
:10EB140049040840009A02219140884205D1019895
:10EB24000168486802221043486001990120087175
:10EB340001990020487102A90020087002A80078F9
:04EB440003B0704763
:10EB480085B00490039102920193002000900498EC
:10EB5800006800900398002805D102980099401891
:10EB68000830009004E00298009940181430009092
:0CEB7800019800990860002005B070476B
:10EB840083B0029001A801806846027000780028D2
:10EB940004D001A800880299886103E001A80088D4
:08EBA4000299886203B070477A
:10EBAC0083B0029001A80180029949690091009AF2
:10EBBC00018810460840000491434018029988616E
:04EBCC0003B07047DB
:08EBD00081B0009001B0704714
:08EBD80081B0009001B070470C
:08EBE00081B0009001B0704704
:08EBE80081B0009001B07047FC
:10EBF00085B00490039102920498006A00900499F1
:10EC0000086A012290430862049880690190019883
:10EC1000F021884301900298010101980843019076
:10EC200000980A21884300900399009808430090B7
:10EC300001980499886100980499086205B07047AA
:10EC400085B00490039102920499086A10229043BF
:10EC500008620498806901900498006A0090019805
:10EC60000F2109038843019002980103019808438A
:10EC700001900098A021884300900398010100981A
:10EC800008430090019804998861009804990862EB
:04EC900005B0704714
:08EC940081B0009001B070474F
:08EC9C0081B0009001B0704747
:08ECA40081B0009001B070473F
:10ECAC008AB00390039884214058212852D10398AC
:10ECBC006A21405A02A9088002A80088002849D07D
:10ECCC0003985621405A00282AD1EFF31080059062
:10ECDC000598019001220992099880F310880398F5
:10ECEC0001688868D205904388600198089008985C
:10ECFC0080F31088EFF310800490049800900120AA
:10ED0C000790079880F310880398016808684022E0
:10ED1C001043086000980690069880F3108819E05C
:10ED2C0003980068C069000600280ED50399086D89
:10ED3C000078096888620399086D401C086503997E
:10ED4C005622885A401E8852FFE70298401E02A99C
:08ED5C000880B1E70AB070471E
:08ED640081B0009001B070477E
:0CED6C0082B001906846018002B0704740
:08ED780081B0009001B070476A
:08ED800081B0009001B0704762
:10ED880083B0019001988021405C012803D102A939
:10ED98000220087026E001998022012088540199F8
:10EDA8008422242088500198006800680090019807
:10EDB8000368186801218843186000984907884348
:10EDC8000090019900204866009801990968086038
:10EDD800019920208850019980220020885402A996
:0CEDE8000020087002A8007803B07047FB
:10EDF40000B583B0029001A8017002988068009069
:10EE04000098401C0299496888420CD801980299DC
:10EE14000968009A88540098401C029988600299F5
:10EE2400C868401CC860029988684968884211D142
:10EE3400029A106911689268FEF770F9029989685C
:10EE4400884204D002990020C043C86002E00299BD
:08EE54000020886003B000BD3E
:08EE5C00C1174840401A70473D
:10EE6400010002000400060008000A000C00100063
:08EE74002000400080000001B5
:10EE7C0043616E6E6F74207265616420737461748B
:10EE8C0069737463616C20646174612066726F6D68
:0FEE9C0020464C415348206D656D6F72792100FF
:10EEAB004144432063616C6962726174696F6E20C7
:07EEBB006572726F72210005
:10EEC2005374617274696E6720566563746F722041
:10EED2005461626C6520636F7079696E6720667237
:10EEE2006F6D20464C41534820746F2052414D2E85
:03EEF2002E2E00C1
:10EEF5004D6F646520302069732073656C6563749C
:10EF050065642E204175746F2D7265636F6E6E6535
:0BEF15006374206973204F46462E00F5
:10EF20004D6F646520312069732073656C6563746F
:10EF300065642E204175746F2D7265636F6E6E650A
:0BEF40006374206973204F46462E00CA
:10EF4B004D6F646520322069732073656C65637443
:10EF5B0065642E204175746F2D7265636F6E6E65DF
:0BEF6B006374206973204F46462E009F
:10EF76004D6F646520332069732073656C65637417
:10EF860065642E204175746F2D7265636F6E6E65B4
:0BEF96006374206973204F46462E0074
:10EFA1004D6F646520342069732073656C656374EB
:10EFB10065642E204175746F2D7265636F6E6E6589
:0BEFC1006374206973204F46462E0049
:10EFCC004D6F646520352069732073656C656374BF
:10EFDC0065642E204175746F2D7265636F6E6E655E
:0BEFEC006374206973204F46462E001E
:10EFF700555020627574746F6E206973206C6F6E44
:0BF00700672D707265737365642E0046
:0BF0120056613A20253664206D560040
:0BF01D0056623A20253664206D560034
:0BF028004441435F413A20253464005E
:0BF033004441435F423A202534640052
:03F03E004F500030
:03F04100434C003D
:03F0440042410046
:03F0470041420043
:03F04A002573002B
:03F04D004F54001D
:03F050004F43002B
:03F053004F4C001F
:03F056004C420029
:10F0590043757272656E742063616C6C696272616A
:10F0690074696F6E2073657175656E63652073745D
:07F0790061727465642E0052
:10F08000095B2534645D2053616D706C6564207686
:0BF09000616C75653A202534640A00AD
:0BF09B0048414C206572726F7221002A
:10F0A60053415645204C4F434B2D4B455920434F1A
:07F0B6004D4D414E442E00B8
:10F0BD0043616E6E6F7420726573746F7265206438
:10F0CD00656661756C742073657474696E67732001
:10F0DD0066726F6D20464C415348206D656D6F72A1
:03F0ED0079210086
:03F0F0003A2000C3
:10F0F3004465766963652049443A2053544D33325D
:10F1030047304231206F722053544D3332473043DE
:02F113003100C9
:10F115004465766963652049443A2053544D33323A
:10F1250047303731206F722053544D3332473038D2
:02F135003100A7
:10F137004465766963652049443A2053544D333218
:10F1470047303531206F722053544D3332473036B4
:02F15700310085
:10F159004465766963652049443A2053544D3332F6
:10F1690047303331206F722053544D333247303496
:02F17900310063
:10F17B004672656520737061636520666F722063EC
:10F18B006F66696775726174696F6E20696E206650
:10F19B00616B6520454550524F4D3A2025752062D5
:06F1AB00797465730A008F
:10F1B1004D41585F504F535349424C455F44494676
:10F1C100465F544F5F4D4541535552453A20257591
:02F1D1000A0032
:10F1D30043616E6E6F742073746172742041444393
:0EF1E30020696E20444D41206D6F646521004F
:10F1F10043616E6E6F7420636F707920566563741E
:10F201006F72205461626C652066726F6D20464C8E
:10F2110041534820746F2052414D2120444D4120DB
:0EF221006973206E6F7420726561647921003C
:10F22F0043616E6E6F742066696E69736820636FD9
:10F23F007079696E6720566563746F7220546162CE
:10F24F006C652066726F6D20464C41534820746F79
:06F25F002052414D210088
:10F265004D6F646520302069732073656C65637428
:10F2750065642E204175746F2D7265636F6E6E65C2
:0AF285006374206973204F4E2E00C1
:10F28F004D6F646520312069732073656C656374FD
:10F29F0065642E204175746F2D7265636F6E6E6598
:0AF2AF006374206973204F4E2E0097
:10F2B9004D6F646520322069732073656C656374D2
:10F2C90065642E204175746F2D7265636F6E6E656E
:0AF2D9006374206973204F4E2E006D
:10F2E3004D6F646520332069732073656C656374A7
:10F2F30065642E204175746F2D7265636F6E6E6544
:0AF303006374206973204F4E2E0042
:10F30D004D6F646520342069732073656C6563747B
:10F31D0065642E204175746F2D7265636F6E6E6519
:0AF32D006374206973204F4E2E0018
:10F337004D6F646520352069732073656C65637450
:10F3470065642E204175746F2D7265636F6E6E65EF
:0AF357006374206973204F4E2E00EE
:10F36100555020627574746F6E20697320707265D8
:06F37100737365642E00B9
:02F377004E0046
:06F37900523A202573004A
:02F37F000A0082
:10F3810043616E6E6F742073617665206461746190
:10F3910020696E20464C415348206D656D6F72792E
:02F3A100210049
:0EF3A3004E4D49204552524F522121210A0061
:02F3B1000A0050
:05F3B3004D41494E0030
:10F3B80043616E6E6F742073746172742054494D8A
:05F3C800455232210056
:05F3CD001B5B324A0049
:10F3D20050726F6772616D20737461727465642E0E
:01F3E200002A
:10F3E30043505520467265713A20257520487A0AA4
:01F3F3000019
:10F3F40043616E6E6F74207265616420636F6E6624
:10F40400696775726174696F6E2066726F6D2046EC
:0DF414004C415348206D656D6F72792100E9
:10F42100257325733A204144432043616C6962721C
:10F431006174696F6E2076616C75653A2025750A75
:01F4410000CA
:10F4420043616E6E6F742073746F70204144432168
:01F4520000B9
:10F4530025733A204441432043616C6962726174AD
:10F46300696F6E2076616C756520666F72206368C4
:0DF47300616E6E656C20313A2025750A002F
:10F4800025733A204441432043616C696272617480
:10F49000696F6E2076616C756520666F7220636897
:0DF4A000616E6E656C20323A2025750A0001
:10F4AD0049742069732074696D6520746F207361D0
:10F4BD00766520737461746973746963616C20641B
:10F4CD0061746120696E20466C617368206D656D95
:05F4DD006F72792E00A2
:10F4E200496C6C6567616C204D6F6465206973209F
:10F4F20073656C65637465642E2044656661756C22
:10F5020074204D6F646520342069732073656C65C7
:10F51200637465642E204175746F2D7265636F6E1E
:0DF522006E656374206973204F46462E000D
:05F52F002573257300A7
:09F53400493A202535642041000C
:09F53D004F56503A2025317300AD
:09F546004C56503A2025317300A7
:0DF54F00543A202532642E256420B043007C
:10F55C00095B2534645D2053616D706C65642076A5
:10F56C00616C7565733A20492B203D20253675203A
:0DF57C00202020492D203D202536750A0055
:10F5890009094F66667365742076616C7565733A0F
:10F5990020492B203D20257520202020492D203D64
:05F5A9002025750A0099
:10F5AE0009094F66667365742076616C75653A203D
:05F5BE002534640A0081
:10F5C300556E6B6E6F776E20636F6D6D616E642128
:01F5D3000037
:0DF5D4005553415254206572726F72210030
:10F5E10025733A205265766973696F6E206E756D69
:0CF5F1006265723A2030782534580A0018
:10F5FD004672656520737061636520666F72207356
:10F60D0074617469737469637320696E2066616BCC
:10F61D006520454550524F4D3A202575206279742D
:04F62D0065730A00F7
:10F63100435055207370656564206973206E6F7443
:08F641002036344D487A210007
:10F6490046697273742073746172742120577269E8
:10F6590074696E672064656661756C7420636F6E8A
:0CF6690066696775726174696F6E21003C
:08F675001B5B313B33326D00D9
:10F67D00566563746F72205461626C6520686173A6
:10F68D00206265656E20636F706965642066726FB8
:10F69D006D20464C41534820746F2052414D2E0031
:10F6AD00496C6C6567616C204D6F646520697320D2
:10F6BD0073656C65637465642E2044656661756C55
:10F6CD0074204D6F646520342069732073656C65FB
:10F6DD00637465642E204175746F2D7265636F6E52
:0CF6ED006E656374206973204F4E2E0080
:10F6F900444F574E20627574746F6E206973207081
:08F709007265737365642E0044
:08F711001B5B323B33306D003D
:08F719002573207C20257300FC
:0CF721005661623A20253464206D5600C9
:0CF72D005662623A20253564206D5600BB
:10F739001B5B323B33316D591B5B313B33326D00FF
:08F749001B5B313B33316D0005
:08F751001B5B313B33366D00F8
:08F75900434847202D20310038
:08F76100434847202D20300031
:10F769000909566F6C746167652D64726F70204169
:10F7790044432076616C75653A202535642E0A006C
:10F7890009090946696E616C20766F6C7461676559
:10F799002D64726F70204144432076616C75653A1F
:10F7A900202534752E2046696E616C20766F6C7445
:10F7B9006167652D64726F702076616C75653A209A
:08F7C900253375206D560A007E
:10F7D10043616E6E6F742073617665206E6577206C
:10F7E100534E20696E20464C415348206D656D6F24
:04F7F1007279210008
:10F7F50043616E6E6F742073746172742054494D49
:10F80500313720696E20495352206D6F64652100A0
:08F815001B5B313B33316D0038
:10F81D00486172646661756C74204552524F522175
:04F82D0021210A008B
:08F831001B5B323B33326D001A
:08F839001B5B323B33336D0011
:08F841001B5B323B33316D000B
:04F849004D4F4400DB
:08F84D000101010307010000A5
:08F8550008040204080101018E
:10F85D0030313233343536373839414243444546F9
:03F86D00FFFFFF9B
:10F87000911E0108ED050020490E0000A31E01089D
:10F8800000000020A0F80008ED050000A31E0108FC
:10F89000006000208DFE0008002000003FD200081C
:10F8A00082B00E480168C96A01910068006B00903F
:10F8B00001980F2802D301980F38019000980F2863
:10F8C00002D300980F380090019804490A689060AC
:10F8D00000980968486102B07047C046A81100202E
:10F8E00082B010480168C96A01910068006B0090FD
:10F8F0000198FF210901884202D801980F30019038
:10F900000098FF210901884202D800980F3000902A
:10F91000019804490A68906000980968486102B03B
:10F920007047C046A811002082B00E480168C96A1D
:10F9300001910068006B009001980F2802D3019894
:10F940000F38019000980F2802D300980F380090CC
:10F95000019804490A68906000980968486102B0FB
:10F960007047C046A811002082B010480168C96ADB
:10F9700001910068006B00900198FF210901884205
:10F9800002D801980F3001900098FF2109018842A8
:10F9900002D800980F300090019804490A689060DE
:10F9A00000980968486102B07047C046A81100205D
:10F9B00082B00E480168C96A01910068006B00902E
:10F9C00001980F2802D301980F38019000980F2852
:10F9D00002D300980F380090019804490A6890609B
:10F9E00000980968486102B07047C046A81100201D
:10F9F00082B010480168C96A01910068006B0090EC
:10FA00000198FF210901884202D801980F30019026
:10FA10000098FF210901884202D800980F30009019
:10FA2000019804490A68906000980968486102B02A
:10FA30007047C046A811002082B01D480068C06A07
:10FA400001901C4800681C493A22895E40181B49F5
:10FA5000884206DC01980F2802D301980F380190E4
:10FA600010E01448006814493A22895E401814498D
:10FA7000884207DB0198FF210901884202D80198DA
:10FA80000F30019001990A48026891600068006B8C
:10FA900000900098FF210901884202D800980F3099
:10FAA0000090009802490968486102B07047C0465A
:10FAB000A811002018120020101300205109000086
:10FAC0005309000082B01D480068006B01901C487B
:10FAD00000681C493A22895E40181B49884208DCAC
:10FAE0000198FF210901884202D801980F30019046
:10FAF0000EE01348006813493A22895E4018134902
:10FB0000884205DB01980F2802D301980F38019035
:10FB100001990A48026851610068C06A0090009823
:10FB2000FF210901884202D800980F300090009808
:10FB300002490968886002B07047C046A8110020D9
:10FB40001812002010130020AB060000AD060000C4
:10FB500082B00E480168C96A01910068006B00908C
:10FB600001980F2802D301980F38019000980F28B0
:10FB700002D300980F380090019804490A689060F9
:10FB800000980968486102B07047C046A81100207B
:10FB900082B010480168C96A01910068006B00904A
:10FBA0000198FF210901884202D801980F30019085
:10FBB0000098FF210901884202D800980F30009078
:10FBC000019804490A68906000980968486102B089
:10FBD0007047C046A81100207047010180B500F0B1
:10FBE0008BF880BD10B584B01E48029000891E4974
:10FBF00008801E480068804702998A881C48026075
:10FC00004A891C490A601C4B1A68022422431A6064
:10FC100000680968884203DB15480068019002E02B
:10FC200014480068019001980390039813494022FA
:10FC3000895E884210D3039A1148016889180160CF
:10FC4000006810490968884205D90F480068804754
:10FC50000B490020086002E009490020086004B058
:10FC600010BDC0462214002018120020741200207B
:10FC70001C1200202012002004000240101300205B
:10FC8000D81200201C0500209412002080B500F03E
:10FC90003BF80C2000F040F80B490C4808600C4879
:10FCA000006800280ED10B49012008600A49096844
:10FCB0000A4A11600A4A41218B00D15A491CD1528B
:10FCC0000849086080BDC046741200203903002036
:10FCD00024120020281200200C12002018050020F9
:10FCE000101300201412002080B5024800F01CF808
:10FCF00080BDC046F40D002008B4024B9C4608BCF1
:10FD00006047C0467182000808B4024B9C4608BC9C
:10FD10006047C046495A000808B4024B9C4608BCDC
:10FD20006047C046B5D8000808B4024B9C4608BCE2
:10FD30006047C0464172000888B00590049103A94D
:10FD400000200870059802900498019015490868F1
:10FD50000122920410430860EFF310800690069889
:10FD6000009072B603A800783F280ED8019800686A
:10FD7000029908600198001D01900298001D0290F0
:10FD80000398401C03A90870ECE707480068C0030B
:10FD9000002800D5F9E700980790079880F31088AD
:10FDA00008B07047142002401020024004000000F8
:10FDB000FFFFFFFFC0E0FFFFC0E0FFFFFFFFFFFF0F
:10FDC0000024F4000100000001000000FFFFFFFF1D
:10FDD00001000000FFFFFFFF01000000FFFFFFFF29
:10FDE00001000000B80B000000DC0500020000006C
:10FDF00001000000040000000100000002000000FB
:10FE000001000000000000000202000000000002EB
:10FE100002020202010000000000000000000000D9
:10FE200000010101000101000100020201010000C6
:10FE300000000000000000000000000000000000C2
:10FE400000000000000000000000000000000000B2
:10FE500000000000000000000000000000000000A2
:10FE60000000000000000000000000000000000092
:10FE70000001010101000101000000010101010078
:10FE800000000000000000000000000000CDCDCD0B
:10FE9000CDCDCDCDCDCDCDCDCDCDCDCDCDCDCDCD92
:10FEA000CDCDCDCDCDCDCDCDCDCDCDCDCDCDCDCD82
:10FEB000CDCDCDCDCDCDCDCDCDCDCDCDCDCDCDCD72
:10FEC000CDCDCDCDCDCDCDCDCDCDCDCDCDCDCDCD62
:020000040801F1
:101E8000CDCDCDCDCDCDCDCDCDCDCDCDCD000000E9
:101E9000206861680834002200E042540139FCD512
:021EA000704789
:101EA20020686168A2680C3401E08B5C8354013ABB
:041EB200FBD57047A5
:101EB600FFFFFFFFFFFFFFFFFFFFFFFFFFFFFFFF2C
:101EC600FFFFFFFFFFFFFFFFFFFFFFFFFFFFFFFF1C
:101ED600FFFFFFFFFFFFFFFFFFFFFFFFFFFFFFFF0C
:101EE600FFFFFFFFFFFFFFFFFFFFFFFFFFFFFFFFFC
:06EFF600FFFFFFFFFFFF1B
:04EFFC00D0C9B07A4E
:040000050800D35FBD
:00000001FF
